:1000000082C400000C94C831B6C40000B4C400001F
:10001000B2C40000B0C40000AEC40000ACC4000014
:10002000AAC40000A8C400000C94FE2F0C94E63073
:100030000C94B32FA0C400009EC400009CC4000018
:100040009AC4000098C4000096C4000094C4000044
:1000500092C400000C94DA2F8EC400008CC40000FF
:100060008AC4000088C4000086C4000084C4000064
:1000700082C4000080C400007EC400007CC4000074
:100080007AC4000078C4000076C4000074C4000084
:1000900072C4000070C400006EC400006CC4000094
:1000A0006AC4000068C4000066C40000050109803D
:1000B000A101850319012AB700150126B700950192
:1000C00075108100C0050C0901A101850419012AE0
:1000D000A002150126A002950175108100C00660DE
:1000E000FF0961A1010962150026FF00952075082E
:1000F00081020963150026FF00952075089102C052
:1001000005010906A101050719E029E715002501E8
:10011000950875018102950175088101050719008F
:1001200029FF150026FF00950675088100050819AE
:1001300001290515002501950575019102950175A7
:10014000039101C00000000000000000000000005A
:10015000000000000000000000000000000000009F
:1001600000000000000000007E0F00D4FFFFFFC76A
:100170000000007800000000000000002A2B28008A
:100180000000000000000000000000000000002946
:10019000000000002C1E3420212224342627252E86
:1001A000362D3738271E1F202122232425263333BE
:1001B000362E37381F0405060708090A0B0C0D0EEA
:1001C0000F101112131415161718191A1B1C1D2FB6
:1001D0003130232D350405060708090A0B0C0D0ED6
:1001E0000F101112131415161718191A1B1C1D2F96
:1001F0003130354C09025B00030100A0FA0904000C
:10020000000103010100092111010001224400073E
:100210000581030800010904010002030000000930
:10022000211101000122220007058203200001079D
:100230000503032000010904020001030000000976
:100240002111010001223200070584032000011260
:100250000100020000000810CB57531005010203F3
:10026000011C037600690061006C003A00660036EC
:10027000003400630032006200330063000000229B
:10028000035100750065006600720065006E006332
:1002900000790020005200650076002E0020003515
:1002A0000000000E034B0065006500620069006FEE
:1002B000000000040309043A003B00167C1E001FE6
:1002C0000020002100220023003C003D002B0014F0
:1002D000001A0008001500170000003E003F00391A
:1002E0000004001600070009000A00000040004159
:1002F00000E10000001D001B00060019000500427F
:10030000004300E000E200E300215200002C000066
:100310000024002500260027002D002E004C002A76
:10032000004A001C0018000C00120013002F0030BF
:100330000031004D000B000D000E000F00330034A3
:1003400000000028004B0011001000360037003874
:10035000000000E50052004E0021522C00E600E4AF
:1003600000E7000000500051004F0001000100169E
:100370007C3A003B003C003D003E003F0001000194
:1003800000207821780100520001000100000001E6
:1003900000010001000100500051004F0001000069
:1003A0000001000100010000000100010001000146
:1003B0000001000100010035020100010001000000
:1003C000000100000040004100420043004400459D
:1003D000004C002A000100010001000100010001A1
:1003E0000001000100010001000100010001000105
:1003F00000010001000000010001000100010001F6
:1004000000010001000000010001000100010001E5
:10041000000100010001000000010001000100AA2C
:1004200000A9004E004B0022782178AC00AB0022DE
:1004300023252628292A2C2D2F3032333536383AD9
:100440003B3D3E4042434547494A4C4E505153552F
:1004500057595A5C5E6062646668696B6D6F717350
:100460007577797B7D7F81838587898A8C8E909251
:100470009496989A9C9E9FA1A3A5A7A8AAACAEAF5C
:10048000B1B3B4B6B8B9BBBCBEBFC1C2C3C5C6C7A1
:10049000C9CACBCCCDCED0D1D2D2D3D4D5D6D7D752
:1004A000D8D9D9DADADBDBDBDCDCDCDCDCDDDDDD9A
:1004B000DDDCDCDCDCDCDBDBDBDADAD9D9D8D7D796
:1004C000D6D5D4D3D2D2D1D0CECDCCCBCAC9C7C643
:1004D000C5C3C2C1BFBEBCBBB9B8B6B4B3B1AFAE81
:1004E000ACAAA8A7A5A3A19F9E9C9A989694929027
:1004F0008E8C8A89878583817F7D7B7977757371FF
:100500006F6D6B6968666462605E5C5A59575553DB
:1005100051504E4C4A4947454342403E3D3B3A3894
:1005200036353332302F2D2C2A292826252322FF39
:10053000AA7F55400102030C0D0E0F0007060504AB
:100540000B0A090800010101010101010101020278
:100550000202020202020203030303030303030471
:10056000040404040404050505050506060606063C
:10057000070707070708080808090909090A0A0AF6
:100580000B0B0B0C0C0C0D0D0D0E0E0E0F0F0F1098
:100590001011111112121313141415151616171722
:1005A000181819191A1A1B1B1C1D1D1E1E1F20208E
:1005B000212222232424252626272829292A2B2CD8
:1005C0002D2D2E2F30313232333435363738393AFB
:1005D0003B3C3D3E3F404142434445464748494AF3
:1005E0004C4D4E4F50515354555658595A5B5D5EC1
:1005F0005F616264656668696B6C6D6F707273755C
:1006000077787A7B7D7E8082838587888A8C8E8FBF
:1006100091939596989A9C9EA0A2A3A5A7A9ABADED
:10062000AFB1B3B5B7BABCBEC0C2C4C6C9CBCDCFDB
:10063000D1D4D6D8DBDDDFE2E4E7E9EBEEF0F3F589
:10064000F8FAFDFF1E0F0500047F3F1F643214649B
:100650003214783C1E1E140A05FD377A585A0000E1
:1006600004E6D6B4460200210116000000742FE50E
:10067000A3E0078302415D003D8889C65436C31755
:100680004FE4E5014D6F8DD6A60C93036C2ABA3268
:100690000B67D074BE2E4BF24146C9FCB1ED076426
:1006A000B2A6D1E77F01123412D844B38A29E88573
:1006B0007D499BF3C5C6F93A621903EF4B160E83C9
:1006C000D9D372903FAE672D67FEA90D0C2B555004
:1006D000C5F4F26742EB0EE072E3BADDF91AF2CE2E
:1006E000877476FD39CD8DBC4C888B38449B2FC2E6
:1006F000F1DFCA31665673B11BBB58ED7F9D22C531
:100700009DF7AEE69F227067697C01303948E2E0D0
:1007100090DA9E3164190800215D2B206243A131DB
:10072000635CB4CB03F024A60CDEF21B4926030065
:10073000724711A63CE5B5F6562A4E40E9EE762EF4
:10074000C66361CC27EC9B9EAD7D453D67C15D775F
:100750003F51AAD03FF712125DC77E306B1DCAA46D
:100760008F6758B28F0CC7B4530B1E19C15542AFD7
:10077000A0C9DF24B562F99A78DF81CAF8CA01BD41
:10078000C29321823C940BCE04DEE007A67975115A
:100790005B3C911506DC15D72BD5199BCD8DBEABD7
:1007A000C34D67C7E51D321E17B34413C41D6058FF
:1007B000D37E621EEF4B1B516D4A0B3C3A4FA2A2F7
:1007C000B33F487C06DDF44E9595928332BBEFA390
:1007D00014F1194290E5ACC12BF36694979C6F2BF2
:1007E0000D15920D19516BB81F7CDC33E2B0C16A54
:1007F0002116AB933BBEF0DB7F1AABED92C7908323
:100800007AA4E80DF1F8C4866E6F064A108A0535A1
:10081000E24210ACB1487A6344E6A75539C232319E
:10082000075841A1B197EC749B847A21707B804971
:10083000FC95849409D2F5F3BC7864C3DDCC2154D3
:10084000458E6517084EEBE5BBE82E5B5095E28CB4
:10085000B2F5CAD3D79239C6BAE1F6CF0028323AF8
:1008600080F59F24E0DE66BD8D699A5EDADB410F7C
:1008700016ED364D63B0B13AA81393C879CDABE10C
:1008800021CBC4239F263CD4188AA53CA6C4901F24
:100890002B3768AF5BFF261046C117C57A0135D9E3
:1008A0009DDDC940F41E88CD5348AC907192846E92
:1008B0002B3420CF118065A88700000000FFB37B98
:1008C000C8DD56ED380001DD04840F0000BD1B12A9
:1008D000F1B1C467FB020000000004595A504F52A6
:1008E000514A4D4B4E2A4C2F30B6B7ABACBBBCA9CE
:1008F000AABDBE0D0E0B0F1A050805090507181134
:10090000130408120C0011241FBECFEFDAE0DEBF83
:10091000CDBF04B603FE18C08091A1049091A2043B
:10092000A091A304B091A4048730904BA740B04B92
:1009300059F41092A1041092A2041092A3041092F0
:10094000A404E0E0F8E3099524E0A2E4B2E001C0E9
:100950001D92A13AB207E1F712E0A0E0B1E0E6E4AF
:10096000FAE602C005900D92A234B107D9F70E94B1
:10097000F7270C94EB3444CB9C01FB019A9581152D
:100980009F4120F5832F8170B32FB270AA27732F58
:1009900074706627532F5870442734FF0DC082951A
:1009A000807FAB2B09F08062672B09F08064452BB8
:1009B00009F0806809950895AB2B09F08260672BD8
:1009C00009F08460452BB1F38860F4CF80E0F2CF6A
:1009D0000C9447330895982F92959F7024E09111BD
:1009E00002C020E0982F892F86958695811511F0F9
:1009F0002E5F982F892F8695820F08958093440447
:100A0000089580934504089521E030E001C0220F4D
:100A10008A95EAF780914504822BF3CF21E030E0FC
:100A2000A90102C0440F551F8A95E2F7CA018095BB
:100A3000909145048923E5CF9B01677091E001C047
:100A4000990F6A95EAF763E0369527956A95E1F77D
:100A5000B901660F771F260F371FFA01E20FF31F48
:100A600040E050E0682F70E08191DF019B01042E8F
:100A700002C0369527950A94E2F721702195282720
:100A8000292328272E934F5F5F4F4330510561F78D
:100A900008959C01A82FA77083E0369527958A9525
:100AA000E1F7C901880F991F820F931FFB01E80F1F
:100AB000F91F40E050E080E0219130E00A2E02C0B2
:100AC000369527950A94E2F721703327042E01C04A
:100AD000220F0A94EAF7822B4F5F5F4F4330510594
:100AE00059F70895282F862F903F71F09A3068F4B7
:100AF000293050F4622F70E029E0929F600D711D43
:100B000011244DEA53E098CF08959C5F9230E0F7AE
:100B1000622F70E04AEA53E0F6CF903FB9F09A3086
:100B200070F4893098F4282F30E06DEA73E0A90161
:100B3000E9E09E9F400D511D1124CA01AACF9C5F80
:100B4000923020F46AEA73E090E0F8CF80E00895F4
:100B50009091450421E030E0F90101C0EE0F8A9543
:100B6000EAF7D90102C0AA0FBB1F6A95E2F7EA2B88
:100B700001C0220F4A95EAF7892F8E23E81303C09C
:100B8000892F822B3ECF2095822F8923FBCF809106
:100B90004D0490914C04981301C008958F5F8770A5
:100BA000FACF909147048095892380934704282F9A
:100BB0002770211110C0891771F09091A00492FF45
:100BC0000AC086958695869529DF10924704109273
:100BD0004904109248040895982F909580914204FA
:100BE000892380934204089580914104811531F056
:100BF0001092410410924B0410924A040895803ED2
:100C00009105D9F1C8F48133910509F482C048F403
:100C10008932910509F472C08A32910509F480C0C5
:100C2000089589339105E9F082389105D1F0853333
:100C3000910509F45EC00895843E9105D9F148F408
:100C4000823E910539F1833E910549F181EE90E0B4
:100C50000895863E9105C9F1873E910509F43EC08D
:100C6000089520919F042370211164C02091A00455
:100C700023FF14C089E290E0089520919F0420FD95
:100C800045C03091A00430FF09C024FD24C083EE8C
:100C900090E0089520919F0422FDF7CF08952091C0
:100CA0009F0422FD44C03091A00430FD43C024FFC6
:100CB000F5CF11C02091A00421FFF0CF80919F04B7
:100CC00084FD09C087EE90E0089520919F0423FFE2
:100CD000E5CF24FFF7CF80E090E0089520919F04B6
:100CE00023FD2BC03091A00431FFE1CF84EE90E0D2
:100CF000089520919F0425FFD1CFBCCF20919F0460
:100D000025FD1EC02091A00423FFC8CF89E390E0F9
:100D1000089520919F0426FFC1CF8AE290E00895B4
:100D200020919F0426FFBACF81E390E0089582EEE0
:100D300090E0089580EE90E0089586EE90E00895AA
:100D400085E390E0089590919F0492FF10C041E0E8
:100D5000282F2471243009F040E031E0282F287139
:100D6000283009F030E0431711F02CE0822793FF80
:100D700010C041E0282F2471243109F040E031E017
:100D8000282F2871283109F030E0431711F02CE0AA
:100D900082273091A00430FF10C051E0282F21712C
:100DA000213009F050E041E0282F2871283009F067
:100DB00040E0541711F029E0822731FF10C041E0D4
:100DC000282F2171213109F040E031E0282F2871CE
:100DD000283109F030E0431711F029E0822794FD13
:100DE000877E08951F93CF93DF9309DFEC01811570
:100DF00022E5920708F052C0811540E5940708F0FB
:100E0000CDC0803E910520F58D3C910508F0A1C034
:100E1000883A910570F4853A910508F097C08130C1
:100E20009105B9F10497813A910598F1C0E0D0E0BD
:100E300030C0885A91094B97C8F7C85AD0E0CC0FF8
:100E4000DD1FCB52DE4F0990D881C02DD46421C064
:100E5000811550E49507B0F4C11580E2D80708F079
:100E6000B3C0C83ED105A8F0CE019A9581159F4127
:100E7000E8F68D2F68DF182FCE019927C0DEEC0130
:100E8000D12B07C09927BBDECC27DF70C82BD92B0D
:100E9000D06ACE01DF91CF911F910895803842E54D
:100EA0009407C8F5803652E5950708F05BC0C0345A
:100EB00082E5D807D0F4C03292E5D90708F04BC0DC
:100EC0008C2F8695869520E2829FC0011124C370E5
:100ED00021E030E0A90102C0440F551FCA95E2F796
:100EE000EA01C82BD92BDD68D4CF8C2F8695869547
:100EF000877050E2859FC0011124C37021E030E06B
:100F0000A90102C0440F551FCA95E2F7EA01C82B98
:100F1000D92BDC68BECF803C52E5950758F48F7121
:100F2000C03AD245A0F590E0982F8827EC01C46F15
:100F3000D06AAFCF805C9245809708F077CFDC2FE6
:100F4000CC27CC27DF71C06FD06AA3CFA497D06421
:100F5000A0CFD0659ECFCF71D0E0DC2FCC27C16F62
:100F6000D06A97CF86958695877020E2829FC001D0
:100F70001124C37021E030E0A90102C0440F551FC5
:100F8000CA95E2F7EA01C82BD92BDA6882CFDBDEFB
:100F9000C82FD0E0DC2FCC27D0627BCF8F71D3DE7F
:100FA00093E0CC0FDD1F9A95E1F7CC27DF70282F57
:100FB00030E084FF05C050E1859F90011124332764
:100FC000C22BD32BD06965CF8D2F8F71BCDE182F2C
:100FD000CE01992714DEEC01D12BDECF80E00895FD
:100FE000F894E82FE295EF70F0E041A18F7021E0D6
:100FF00030E0B90102C0660F771F8A95E2F7CB0196
:10100000962F9095942391A392A1892B82A37894F3
:10101000089581E080935D0308950895CF92DF9253
:10102000EF92FF921F93CF93DF93172FE82FF0E0FB
:10103000EC5BFA4F71110CC0E4918E2F7E2F6E2F56
:10104000DF91CF911F91FF90EF90DF90CF900895A7
:10105000E62EF12CC72ED12CF491EF2F86E0689F5D
:1010600090011124CFEFD0E0C901BE010E941A33D4
:10107000AB01EE0CFF1C65E5649FC001659F900D00
:101080001124E81AF90A6E2D660F6E0D7E01EC1818
:10109000FD08FE9DD001FF9DB00D11248B2F169FE2
:1010A00070011124EF2CFF246E01CE18DF087601A9
:1010B000FE9D6001FF9DD00C11247E01E61AF1080F
:1010C000B701169F7001179FF00C1124EF2CFF241D
:1010D000CE19DF09FC9F7001FD9FF00C11247F2DBC
:1010E00043305105C1F02C3F334058F44130510595
:1010F000B1F04230510509F0A2CFEB2F8F2D7F2F99
:101100009ECF4430510571F04630510509F497CF18
:101110007B2F8D2D94CF7D2DEB2F8F2F90CF7F2F79
:10112000ED2D8DCFEF2D7B2FF8CFCF93DF93982F21
:10113000762F842FE901692F71DF472F282FFE01B9
:10114000FF27EC5CFA4FE49180911601E81B8E2F8B
:1011500090E038D3DF91CF910895809138048430A6
:1011600028F4837084608093380408958C3AE8F3FF
:101170008370886AF8CFCF938091380480FF03C0D2
:10118000D9D5CF910895C091180180911901C81740
:10119000B8F7EC2FF0E0EC5CFA4FE4918091160187
:1011A000E81B20E040E060E08E2F90E00BD3CF5FA3
:1011B000ECCF0F931F93CF93DF93D82F162F042FCD
:1011C00080913804C091180180FD14C0DF91CF9147
:1011D0001F910F910895EC2FF0E0EC5CFA4FE49131
:1011E00080911601E81B202F412F6D2F8E2F90E04C
:1011F000E9D2CF5F80911901C81768F3BCDFE6CF51
:10120000CF93DF93EC0120913B049C81892F817067
:1012100090FD822F692F627091FD622F492F4470DB
:1012200092FD422FC6DF8C8190E00196877099274E
:101230008C83DF91CF910895982F762F842F209162
:10124000380420FF07C0692FE9DE962F672F482F4B
:10125000892FAFCF0895CF93DF93EC01E8E3F4E05B
:10126000438162818C81E8DF8C818F5F8C83DF9189
:10127000CF910895E5E3F4E0118282818460828356
:101280000895E8E3F4E080818E7F8083F3DFE5E377
:10129000F4E08281816082836ECFCF93DF93EC0193
:1012A000EC81F0E0E15DFB4F4491E8E3F4E0628122
:1012B0008181C2DF8C818F5F8C83DF91CF91089514
:1012C000EF92FF921F93CF93DF93EC0110E0EE2497
:1012D000EA94F12C60911A01161768F04CDF8C81AA
:1012E0009A8190FF1DC08F5F8C83DF91CF911F91FA
:1012F000FF90EF90089520911801210F3327331F9D
:1013000070E0C7010E942E33962F8C8140913B04E0
:1013100060913A04199F800D112407DF1F5FDACF17
:101320008150E2CFA0E0B0E0E8E9F9E00C94E032CF
:10133000EC018A8101E080FD0FEF8C81811109C0F1
:10134000013019F480911A0181508093F30281E0F9
:101350008C8310E080911A011817B0F00CDF909187
:10136000F302013009F053C080911A0181509115A8
:1013700019F08FEF890F91E08093F3029C83CDB732
:10138000DEB7E9E00C94FC32E0911801E10FF0E0E7
:10139000EC5CFA4FE49180911601E81B20E040E0FC
:1013A00060E08E2F90E00ED294E0E92EF12CB12C6B
:1013B000C12ED12C8091F3028B0D813114F18F70ED
:1013C000082E001C00088C150D04A1F48091180152
:1013D0009601280F311D40913B046E2D6403A0013E
:1013E0001124559547955595479560913A048091FC
:1013F00039049BDEB00E81E0E81AF108D9F61F5FD0
:10140000A9CF87FFDDCF90911A01890FD9CF892FFE
:1014100090E0019660911A0170E00E942E33982F9F
:10142000ABCF1F93CF93DF93EC018C81811109C067
:1014300081E08C831092F20292E0909306018093F7
:1014400005011091180180911901181740F110E061
:1014500060911A01161798F18EDE80910501909126
:10146000F202980F9093F20220910601280F209328
:101470000601121654F420911A012150330B092E43
:10148000001C00089217030634F081958093050133
:10149000813009F41C82DF91CF911F910895E12FD3
:1014A000F0E0EC5CFA4FE49180911601E81B20E03B
:1014B00040E060E08E2F90E085D11F5FC4CFE12F28
:1014C000F0E070E0CF010E942E3320911801280F28
:1014D0008091F20230E0082E001C0008E817F005A9
:1014E0008CF080910601082E001C00088E170F0654
:1014F0004CF040913B0460913A048091390415DE30
:101500001F5FA6CFF901EC5CFA4FE49180911601C0
:10151000E81B20E040E060E08E2F90E053D1F0CF58
:10152000A6E0B0E0E6E9FAE00C94E1328D839E8318
:10153000AD81BE811496FC912F2F30E0D9010E941D
:10154000DC349B01AC010E94AA346B017C0180E277
:1015500090E09C012F1B3109F901A5E5B0E0A7013E
:1015600096010E94AA3469837A838B839C839F01AE
:10157000DF010E945E339B010E9464339B01AC013A
:101580002C0D3D1D4E1D5F1D69817A818B819C81D3
:101590000E94BA34022F30E00A3240F5A901440F0C
:1015A000551F420F531F55954795142F1095F12C39
:1015B00085E5E82EE01A80911A01F81628F1DBDDA6
:1015C000AD81BE8114969C9181E0911519F0903205
:1015D00019F48FEF8093040180910401890FED814C
:1015E000FE8184832696E8E00C94FD3285E590E048
:1015F000821B930BAC01440F551F480F591F57FF17
:10160000D2CF4F5F5F4FCFCF8E2DF1FC802F209137
:1016100018012F0D3327331F412F60913A0485DDC8
:10162000F394C9CF0F931F93CF93DF93EC0100E0A6
:1016300010E090911A010917110564F09CDD8C816E
:1016400090E00196817099278C83DF91CF911F9153
:101650000F9108954C81809118019801280F311D38
:1016600060913A048091390496950917110544F464
:10167000411541F040913B0458DD0F5F1F4FD9CF1A
:101680004115C1F340E0F8CFFB01811520E292073C
:1016900028F4811541E0940738F408959C013052F4
:1016A0002115304348F00895392F94FF02C0329538
:1016B000307F2081232B208399270895462B22FFFA
:1016C0000FC0982F92959F708F70892B962F9295AF
:1016D0009F706F70692B942F92959F704F70492B5C
:1016E000982F9623961309C050E04095509590E0AE
:1016F0004823592381E0452B09F080E0089590911B
:101700002D03292F30E070912E03A9014F5F5F4F09
:10171000437055277417150689F0255D3C4F60FB13
:1017200087F9F90184839F5F937090932D038091D3
:101730002B038F5F80932B0381E0089580E0089551
:1017400090E06115E9F0855E9E4FFC0180818F3F3E
:10175000B1F0E82FE295EF70F0E041A18F7021E049
:1017600030E0B90102C0660F771F8A95E2F7CB011E
:10177000962F9095942391A392A1892B82A30895EB
:10178000845E9E4FE2CF90E06115A9F0855E9E4F8A
:10179000FC0120812F3F91F0E22FE295EF70E05E97
:1017A000F0E0808190E02F7002C0959587952A9592
:1017B000E2F781700895845E9E4FEACF80E008953D
:1017C0006E9A0895FC01EE0FFF1FE80FF91FEE5807
:1017D000FD4F6183408322830895FC01680F791FC8
:1017E0008FEF41E39191892728E030E0982F990FFE
:1017F00087FF09C0892F842721503040B9F7E617A9
:10180000F70781F70895892FF7CF0F931F93CF9391
:1018100001E010E0082E01C0000F0A94EAF7C09121
:1018200040049C2F9023911115C0909147049695E8
:1018300096959695891306C0109247041092490414
:1018400010924804E1D8C027C0934004CF911F9163
:101850000F910895E3D8F7CF909126048902900163
:10186000112437FF03C08093260408952F373105D4
:101870001CF4980F9093260408959C0180E090E05A
:10188000F901E80FF91FE491E41307C091E08927FB
:10189000F901E80FF11D849108950196861780F3F0
:1018A00080E0089580919803811569F0E091A0038C
:1018B000F091A103309739F00190F081E02D30973D
:1018C00011F00995089580E00895A3E0B0E0EBE6FB
:1018D000FCE00C94E7329C018091700290917102BF
:1018E00082179307B1F03093710220937002E09158
:1018F000A003F091A103309761F00084F185E02D01
:10190000309739F083E089833B832A83CE010196A7
:1019100009952396E2E00C940333A3E0B0E0E3E9F9
:10192000FCE00C94E7329C0180916E0290916F0272
:1019300082179307B1F030936F0220936E02E0910B
:10194000A003F091A103309761F00084F185E02DB0
:10195000309739F084E089833B832A83CE01019656
:1019600009952396E2E00C940333809113010895C6
:101970002FB7F89480916A0290916B02A0916C024B
:10198000B0916D022FBF0895962F2091A00422FFE1
:101990000EC0682F660F660F660F692B60934704B1
:1019A00033D8E6DF909349048093480408952CC807
:1019B00090914104292F2823211559F080958923DE
:1019C00080934104811531F0D3DF80934A049093D2
:1019D0004B04089580E090E0F8CF2FB7F894609121
:1019E0006A0270916B0280916C0290916D022FBF20
:1019F00008950F931F9380919803811521F0EDDFD7
:101A00001F910F910895E9DF0091940310919503C0
:101A10002091960330919703600F711F821F931FCF
:101A2000EFCF80919803811509F0A2CFE2DFCB01BF
:101A3000089508950895FC019B01809160029091A2
:101A400061028617970740F0672B29F48091E80020
:101A50008E778093E800C90140E0009741F441117E
:101A600006C08091E80082FF2FC080E00895209199
:101A700054032115A9F12530A9F12091E80023FD97
:101A80002DC02091E80022FDECCF2091E80020FF3E
:101A9000E4CF3091F3002091F200009719F0283044
:101AA000310558F041E02830310509F040E020913F
:101AB000E8002E772093E800D0CF41914093F100C9
:101AC00001972F5F3F4FE9CF80915403811541F07B
:101AD000853041F08091E80083FFC3CF81E0089515
:101AE00082E0089583E0089580915A0287FF13C031
:101AF0008091E80082FF06C08091E8008B77809398
:101B0000E8000895809154038111F2CF08958091E7
:101B100054038115D9F38091E80080FFF8CF8091BC
:101B2000E8008E77ECCF2091E4003091E50095E657
:101B3000A9012091EC00822F817020FF06C08091C6
:101B4000E80080FF06C080E008952091E80022FDB3
:101B50001AC080915403811589F0853089F08091F5
:101B6000EB0085FD0FC02091E4003091E5004217A5
:101B70005307F9F29A95E1F684E0089582E008951A
:101B800083E0089581E00895E8EDF0E080818E7FA4
:101B900080831092E2001092DA001092E100A0EE31
:101BA000B0E08C9181608C9380818F77808319BCA9
:101BB000A7EDB0E08C918E7F8C9380818F7E8083A7
:101BC000109259020895E091A003F091A10330977B
:101BD00039F00284F385E02D309711F060E2099529
:101BE0000895982F9093E900891771F07091EC0097
:101BF0002091ED005091F00021FD09C09F5F9730CA
:101C000089F78093E9000895762F242F50E03091D2
:101C1000EB003E7F3093EB003091ED003D7F309341
:101C2000ED003091EB0031603093EB007093EC00ED
:101C30002093ED005093F0002091EE0027FDDECFC1
:101C40000895A0E0B0E0E7E2FEE00C94E132C8EDD8
:101C5000D0E088818F7E8883E7EDF0E0808181602D
:101C6000808384E082BF81E08093590288818E7FE7
:101C7000888302EE10E0F80110821092DA0081EE03
:101C8000C82ED12CF601108288818F7788838881B5
:101C90008068888388818F7D888319BC1092540363
:101CA0001092580210920C031092570290EEE92EF7
:101CB000F12CF70180818B7F80838881816088830C
:101CC00042E060E080E08DDFF60180818E7F8083DE
:101CD000F801808181608083808188608083F70142
:101CE00080818E7F8083888180618883CDB7DEB7D5
:101CF000E8E00C94FD32E0914D0490914C0429E011
:101D0000E91302C080E00895AE2FB0E02E9FF001ED
:101D10001124E25BFB4F3181361306C0308138134A
:101D200003C03581341304C0FD013196E770E8CF5C
:101D300081E008953EB13F7B2EB120644FB7F89407
:101D400082E792E0FC010196508168E02EB9000024
:101D500000C057FF3EB9550F000000C000C000C0D2
:101D60003EB900C06A9591F752E0823A950751F763
:101D70004FBF8FE594E00197F1F700C00000089590
:101D800081E08093E00080E28093D8001092C90047
:101D90008FE19EE40197F1F700C0000087E090EB2F
:101DA000DC018093A1049093A204A093A304B093B8
:101DB000A40488E19CE00FB6F894A8958093600095
:101DC0000FBE90936000FFCF0F931F93CF93DF93CD
:101DD0008B01EA0190915403943051F58093E9000E
:101DE0008FEF9091E80095FD06C095ED9A95F1F77B
:101DF00000008A95B1F78091E80085FF19C093DE55
:101E0000811111C08091E80085FD06C08091E80035
:101E10008E778093E800F3CFF80181918F01809352
:101E2000F100219779F78091E8008E778093E800A0
:101E3000DF91CF911F910F910895792F603229F48E
:101E400040E250E0682F82E0BFCF0895CF93DF9348
:101E5000D82FC92F48E050E0682F792F81E0B4DFF8
:101E600088E0ED2FFC2FA2E6B2E001900D928A955A
:101E7000E1F7DF91CF910895BC0143E050E084E0A9
:101E8000A3CFA0E0B0E0E7E4FFE00C94DF32F82E4F
:101E9000E92EB62EA72E8A01809156029AE0C92E0D
:101EA000D12C8A3018F0CC24C394D12CC1E0D0E0DE
:101EB0006B2D7A2D8F2D9E2DF8010995811116C05D
:101EC0002196CC16DD0694F0CC9FC001CD9F900DDD
:101ED000900D112420E030E045E34A95F1F7000031
:101EE0002F5F3F4F28173907B9F7E2CFCDB7DEB7DD
:101EF000EAE00C94FB329091A00492FB222720F997
:101F0000281779F080FB92F99093A00460919F04C8
:101F10007091A00484E090E00E94733482E00C94FD
:101F2000D10508951F93CF93DF93962F122F632F20
:101F30008430D8F49A30C8F44930B8F4C42FD0E0D3
:101F4000CC0FDD1F22E1929FC00DD11D112494EB17
:101F5000899FC00DD11D1124CE0189960E9459344C
:101F6000612FCE018A960E945934DF91CF911F9143
:101F700008950F931F93CF93DF93962F142F022F63
:101F8000632F843018F5923008F528E0829FE00135
:101F9000112434E0939FC0011124C80FD91FC750EA
:101FA000DD4F81E084279E01280F311D280F311D50
:101FB000C9010E94593481E090E0111102C083E010
:101FC00090E0602F8C0F9D1F0E945934DF91CF91BC
:101FD0001F910F910895CF93DF93C0914204809198
:101FE0004604C82B809141048115F1F0C1DC209199
:101FF0004A0430914B04821B930B8838934110F0B4
:102000000E94F405D091410420E086E492E0FC01B6
:102010003081019631112F5F32E08C349307B9F78C
:1020200021110E94F405CD2BC093440248E050E0FA
:1020300062EA73E084E492E00E940B34892BB9F0E9
:1020400088E0E4E4F2E0A2EAB3E001900D928A9520
:10205000E1F7E091A003F091A103309741F00280F5
:10206000F381E02D309719F084E492E00995DF9137
:10207000CF91089510924204E6E4F2E086E0DF0199
:102080001D928A95E9F780E090E01FDC80E090E007
:1020900044DC109246049FCFEDDF2FEF84E39CE0F9
:1020A000215080409040E1F700C0000088E19CE0B2
:1020B0000FB6F894A895809360000FBE90936000CF
:1020C000FFCFAAE2B0E0E7E6F0E10C94E6328AE561
:1020D00092E0FC0101962091F100208322E08236FB
:1020E0009207B9F780915B02893009F457C0C8F4B0
:1020F000823009F4B2C0833009F482C0813081F1AA
:102100008091E80083FFE6C080915A0290915B02C3
:102110009A3008F0DFC0E92FF0E0E351FB4C0C945B
:1021200041338A3009F489C08B3051F780915A02CB
:10213000813231F780915E0290915F02892B01F725
:102140008091E800877F8093E800CEDC81E0909169
:102150005C02911101C080E0809314018BDFD0CF2D
:1021600080915A02813A61F68091E800877F8093DE
:10217000E80080915E0290915F02892B59F060E047
:1021800080E090E070E057DC8091E8008B778093EE
:10219000E800B6CF68E082E692E0F4CF80915A0280
:1021A000813209F0ADCF80915E0290915F028D7F08
:1021B000892B09F0A5CF8091E800877F8093E80004
:1021C0008091E80082FF17C09091F3008091F200A7
:1021D000029731F48091F100813011F0863021F4C2
:1021E0008091F100809313018091E8008B778093B8
:1021F000E8007ADC85CF809154038111E1CF80CF54
:1022000080915A02813A09F07BCF80915E029091D1
:102210005F02892B09F074CF8091E800877F80935B
:10222000E8008091E80080FFFCCF8091140180934A
:10223000F1008091E8008E77DACF80915A028132E6
:1022400009F05ECF8091E800877F8093E8004CDC46
:1022500080915D028093120153CF80915A02813A9E
:1022600009F04ECF8091E800877F8093E80080914D
:10227000E80080FFFCCF80911201D9CF803889F02F
:10228000823841F580915E028F70873018F5809317
:10229000E9008091EB0085FB882780F91092E90026
:1022A00006C080910C03880F90915702892B909162
:1022B000E800977F9093E8008093F1001092F1007E
:1022C0008091E8008E7723C0811116C080915C0256
:1022D000813009F18091E80083FF0AC08091E80015
:1022E000877F8093E8008091EB0080628093EB0011
:1022F000AA96E3E00C940233823061F780915C028D
:10230000811581F01092E9008091E800877F809329
:10231000E800EADBDFCF81E0933009F080E08093D2
:102320000C03F0CF80915E028F702FEF280F2630C4
:1023300088F68093E9002091EB0020FFE3CF9330F3
:1023400031F48091EB0080628093EB00DBCF9091C1
:10235000EB0090619093EB0021E030E0A90102C016
:10236000440F551F8A95E2F74093EA001092EA0065
:102370008091EB008860E8CF8111ACCF10915C02B6
:102380001F778091E3008078812B8093E300809118
:10239000E800877F8093E800A7DB8091E80080FF5A
:1023A000FCCF8091E30080688093E30083E011110B
:1023B00001C082E0809354038DCF8058823008F0B2
:1023C00089CF80915C0290915D028C3D53E095072E
:1023D00091F583E08A838AE289834FB7F894DE011E
:1023E000139620E03EE051E2E32FF0E050935700D7
:1023F000849120FF03C082958F703F5F8F708A3079
:10240000C0F0895C90E08D939D932F5F243161F73C
:102410004FBF8091E800877F8093E8006AE270E018
:10242000CE01019608DB8091E8008B778093E8006D
:1024300051CF805DE7CF292F33272330310509F4B1
:102440004EC078F52130310509F488C08BE590E065
:10245000E4EFF1E02230310509F03CCF2091E800B3
:10246000277F2093E800209160023091610282175B
:10247000930708F49C0140E02115310509F073C071
:10248000411171C08091E80082FDCDCF809154034D
:10249000811549F2853039F28091E80083FFF2CF4F
:1024A000C2CF80915E0290915F022132310509F422
:1024B00046C02232310509F00DCF8330910508F076
:1024C00009CFFC01EE0FFF1FE457FE4F0190F08192
:1024D000E02D87579E4FDC018C9190E010C09C014D
:1024E0003327823021F12330310568F4232BB9F4EE
:1024F000E3EBF2E0E4918E2F90E0E3EBF2E0009763
:1025000009F4E8CEABCF2330310509F0E3CEE1E6A4
:10251000F2E0E4918E2F90E0E1E6F2E0F0CFE3EA22
:10252000F2E0E4918E2F90E0E3EAF2E0E8CFEFE70B
:10253000F2E0E4918E2F90E0EFE7F2E0E0CF83301D
:10254000910508F0C7CEFC01EE0FFF1FEE56FE4FBF
:102550000190F081E02D89E090E080CF82E190E071
:10256000EFE4F2E07BCF80915403811509F45BCF57
:10257000853009F458CF8091E80083FD54CF8091D5
:10258000E80082FD7FCF8091E80080FF75CF9091B9
:10259000F3008091F2002115310519F08830910582
:1025A00050F041E0089709F040E08091E8008E7714
:1025B0008093E80061CF44914093F100319621501F
:1025C00031090196E8CF803809F084CE8091E80087
:1025D000877F8093E800809158028093F10070CE4D
:1025E000811178CE10915C02123008F073CE809188
:1025F000E800877F8093E8001093580275DA111580
:10260000D9F084E08093540342E061EC81E0E9DAA0
:1026100042E261EC84E0E5DA42E261EC82E0E1DA98
:1026200042E260EC83E0DDDA80915403843051F4BF
:1026300082E0809315014ECE8091E30087FDE1CFCB
:1026400081E0E0CF81E0F5CF0F931F93CF93C82FA8
:10265000811531F18CEF8C0F813A98F506E412E088
:10266000F8018191C81701F122E0EC34F207C9F7B3
:10267000EFEF80E0D8019D918D01C91781F0EF3F08
:1026800019F4911101C0E82F8F5F863099F7EF3F61
:1026900031F00E2E000CFF0BEC5BFD4FC2839BDC78
:1026A000CF911F910F910895E6E4F2E08191C81354
:1026B00002C0DF011E9232E0EC34F307B9F78BDC85
:1026C000D7CF80E28C0F883068F4C77081E090E04B
:1026D00001C0880FCA95EAF7C0914204C82BC09385
:1026E0004204DDCF8BE58C0F833030F42C2F245245
:1026F000330BC901EAD8D4CFC85ACB3188F6EC2FB6
:10270000F0E0EE0FFF1FE55FFD4F8081918105D95D
:10271000C7CF811559F19CEF980F913A60F4E6E428
:10272000F2E09191891302C0DF011E9292E0EC3435
:10273000F907B9F750CC90E2980F983050F48770B1
:1027400091E001C0990F8A95EAF7892F0E94EC0564
:10275000F1CF9BE5980F933018F480E090E0B5C876
:10276000885A8B3118F480E090E0D7C808951F9301
:10277000CF93DF93182FEB0167DF209731F4812F80
:10278000C8DFDF91CF911F9108958FE99FE00197F6
:10279000F1F700C000002197F0CF811531F0909142
:1027A0004204892B8093420416CC0895811519F0B8
:1027B0000E94EC0510CC0895811531F090914604EB
:1027C000892B8093460407CC0895811539F08095B4
:1027D00090914604892380934604FDCB089580910F
:1027E0003104811521F082E2F0DF10923104089566
:1027F000A0E0B0E0EEEFF3E10C94E032EC01888170
:10280000811509F1813009F045C08981813051F489
:102810008A81239660E570E0893311F060E070E012
:10282000A6DFEDCF823021F48A8123960DDFE7CF3A
:10283000833021F48A8123966CDFE1CF843041F02C
:1028400022968111DCCFCDB7DEB7E9E00C94FC32E3
:102850008A81239620E030E09AE0682F6053770B5E
:10286000AB016A30710560F02115310551F3EFE9D4
:10287000FFE03197F1F700C0000021503109F4CF9B
:10288000929FB001939F700D11249A01260F371F5C
:102890008991E3CFE82FF0E0EC58FE4FB490282F59
:1028A00026952695269530E0F901EC59FE4FE490E7
:1028B0008770F12C082E02C0F594E7940A94E2F791
:1028C000E0FAEE24FF24E0F8F901EC5AFE4FC49040
:1028D000D12C082E02C0D594C7940A94E2F7C0FA0E
:1028E000CC24DD24C0F8F901EC5BFE4F049110E02C
:1028F00002C0159507958A95E2F701701127E1143A
:10290000F10411F081EEA0DEC114D10411F086EEC5
:102910009BDE60E070E08B2D2ADFC114D10411F042
:1029200086EEF7DEE114F10411F081EEF2DE01151E
:10293000110521F060E070E08CE219DF21965FCF95
:10294000A1E0B0E0E6EAF4E10C94D732462E1A0199
:10295000522EC32E3701A82E880FBB08C5010E9436
:102960006932D82E811509F46BC0C50133E0880F98
:10297000991F3A95E1F7FC01E85CFE4F2381422F55
:1029800050E0211511F041E050E0885C9E4FFC01C1
:10299000648175816F587C4FCE0101960E94183476
:1029A000F10180809180A280B38017D868197909DD
:1029B0008A099B09643671058105910538F4B301D4
:1029C000C8010E94ED0B99818917D1F1E42C042CE8
:1029D000000CFF08C7010E946932D82E811106C081
:1029E000D12C8D2D2196E2E10C94F332C70123E026
:1029F000880F991F2A95E1F7FC01E85CFE4F2381BF
:102A0000422F50E06216710408F4A301885C9E4FC7
:102A1000FC01648175816F587C4F852D9C2D0E942F
:102A20001834B301C8010E94ED0B99818913D8CFE6
:102A30000E94ED0CF1016083718382839383D1CF77
:102A4000A301B801852D9C2D0E941834CACFAAE09D
:102A5000B0E0EDE2F5E10C94E1326B018AE0E82EA2
:102A6000F12C02E713E09E012F5F3F4F4DE653E04C
:102A700061E080E065DF811549F09AE0FE01319662
:102A8000A3E6B3E001900D929A95E1F79AE0E3E6B0
:102A9000F3E0D60101900D929A95E1F72A96E8E0CD
:102AA0000C94FD32A8E0B0E0E8E5F5E10C94E332E7
:102AB00088E0E82EF12C0DE713E09E012F5F3F4FD9
:102AC0004FE553E063E082E03BDF182F811589F189
:102AD00090917C0380915E03981759F100E09091EA
:102AE000800380917F038917F1F0E92FF0E0EB5824
:102AF000FC4F848587FB662760F99F5F93709093F6
:102B0000800390917E039F5F90937E038F770E9456
:102B10007F0B082F8111E3CF84E090E00E9469329F
:102B2000102F182302C00111F7CF80917C038093EE
:102B30005E03812F2896E6E00C94FF32CF92DF925D
:102B4000EF92FF921F93CF93DF9300D000D0CDB7C9
:102B5000DEB7C0905903D0905A03E0905B03F09029
:102B60005C030E94ED0C6C197D098E099F0911E030
:102B7000643671058105910578F10E94F90CDC013C
:102B8000CB010296A11DB11D89839A83AB83BC83BF
:102B900080916101909162018F589C4F209160015A
:102BA000422F50E0253010F044E050E0BE016F5F4E
:102BB0007F4F0E94183485E090E00E946932182F00
:102BC000811551F00E94ED0C6093590370935A03E4
:102BD00080935B0390935C03812F0F900F900F9075
:102BE0000F90DF91CF911F91FF90EF90DF90CF90EA
:102BF00008958F929F92AF92BF92FF920F931F936F
:102C0000CF93DF93CDB7DEB72B970FB6F894DEBF27
:102C10000FBECDBF88E0E8E3F4E08E010F5F1F4FE9
:102C2000D80101900D928A95E1F780913504909139
:102C30003604A091370489879A87AB87F0903704D0
:102C40008090550390905603A0905703B09058037E
:102C50000E94ED0C681979098A099B09E02F312F30
:102C6000643671058105910510F4F11411F180911C
:102C7000690190916A018F589C4F20916801422F01
:102C800050E02C3010F04BE050E06E2F732F0E947C
:102C9000183486E090E00E946932811569F00E9444
:102CA000ED0C6093550370935603809357039093F4
:102CB00058031092370481E02B960FB6F894DEBFCC
:102CC0000FBECDBFDF91CF911F910F91FF90BF90AD
:102CD000AF909F908F9008950F931F93CF93DF93A2
:102CE000843030F56A3020F5493010F5C42FD0E03B
:102CF000CC0FDD1F22E1629FC00DD11D112434EBEA
:102D0000839FC00DD11D1124CE0189960E943834B5
:102D1000082F10E0102F0027CE018A960E94383429
:102D20009801282BC901DF91CF911F910F91089530
:102D300080E090E0F8CFFF920F931F93CF93DF9343
:102D4000F42E843070F5623060F528E0829FE00157
:102D5000112434E0639FB0011124C60FD71FC75060
:102D6000DD4F81E084279E01280F311D280F311D82
:102D7000C9010E943834082F10E0102F002781E08D
:102D800090E0F11002C083E090E08C0F9D1F0E9444
:102D900038349801282BC901CDB7DEB7E5E00C9493
:102DA000003380E090E0F8CF20919C0330919D03A8
:102DB000232BC9F4703F39F4603FA9F480919A0342
:102DC00090919B0308957A3038F4693060F4843030
:102DD00050F4462F672F80CF7D3F41F4623018F4C6
:102DE00041E0843050F080E090E008957C3FD9F7D6
:102DF0006230C8F78430B8F740E09DCFA0E0B0E083
:102E0000E4E0F7E10C94E2327C010091450480910A
:102E10004404082BC3E0D0E010E0C8010C2E02C02F
:102E2000959587950A94E2F780FD09C02197A8F748
:102E3000D12C8D2DCDB7DEB7E7E00C94FE32DC2E21
:102E4000B7018C2FB1DF0E94F206019779F3F1CF21
:102E50000F931F93CF93FC0187819085009789F48E
:102E6000858100811181811581F0611571F0C801A2
:102E7000C5DFC82F682FC8010E947205B8018C2FCA
:102E800093DFCF911F910F910895C8010E948D0586
:102E9000C82FF4CFCF93DF93D82FC92FAFDF6D2F7B
:102EA0007C2F82DF0E94F206DF91CF910895FC0112
:102EB00084818115B1F0878190850097A1F00E94EF
:102EC000F206282F92959F709630B9F080F4925FA9
:102ED0009F70923030F4203FD1F058F481E0283ECA
:102EE00058F080E0089580819181D4DFEACF9A5F25
:102EF000EFCF81E0243FA9F7089591E0813F09F0E9
:102F000090E081E0283E08F080E0892B089581E080
:102F10000895382F292FCB01A32FB22F873B91057E
:102F2000A105B10520F4875B9C4F0C94383480E0F8
:102F3000089585E290E00E943834873D89F486E266
:102F400090E00E9438348E3759F487E290E00E9476
:102F5000383491E08D3209F090E0892F8170089526
:102F600080E0FCCFA6E0B0E0E8EBF7E10C94E232C1
:102F70000BED13E089E1E82E83E0F82E98E0D92EDE
:102F800046E050E0B701CE0101960E942834F801D6
:102F90008D2D11928A95E9F7B8016C5F7F4F898179
:102FA0009A810E94440BF80191838083B8016B5F82
:102FB0007F4F8B819C810E94440BF8019383828315
:102FC0008D8186838E818783F6E0EF0EF11C085F8A
:102FD0001F4F89E4E81683E0F80691F62696E7E0AD
:102FE0000C94FE32A6E0B0E0E8EFF7E10C94DA32A0
:102FF000A0905203B090530381E090E0909353036C
:10300000809352033FE1E32E34E0F32EC12CD12C08
:1030100010E0360100E01AC021E030E0123020F468
:10302000F401859195919C01452D602F812F0E947F
:10303000920F539422E0820E911C39E05312ECCF90
:103040000F5F89E0680E711C0A3049F0C301880FD8
:10305000991FDC01A954BD4F4D01512CDDCF21E05A
:1030600030E0123020F4F701859195919C0141E008
:1030700060E0812F0E94B90F21E030E0123028F487
:10308000F7013296859195919C0140E060E0812F97
:103090000E94B90F21E030E0123028F4F701349695
:1030A000859195919C0141E061E0812F0E94B90FCB
:1030B00021E030E0123028F4F701369685919591A1
:1030C0009C0140E061E0812F0E94B90F1F5FB8E0D2
:1030D000EB0EF11C2AE5C20ED11C143009F099CF79
:1030E000FE01319686E0DF011D928A95E9F709E13C
:1030F00013E07F0146E050E0B801C7010E94773439
:103100000A5F1F4F0934B3E01B07A1F7B0925303C6
:10311000A09252032696EFE00C94F632A0E0B0E0C5
:10312000E4E9F8E10C94D932FC016280448081E04A
:103130008483EFE2F4E07490EEEAF4E0E491C0916D
:103140003B04C695C158D0E0CC0FDD1FCD2FDD2745
:10315000812C25E0922EAA24AA94B12C55245A94AD
:10316000E719EE2EF12C80911A01881638F00E9492
:10317000BB08CDB7DEB7E0E10C94F532C82CD12CFA
:1031800083E0681658F4989CF0011124EE55FD4F29
:1031900080913904808380913A04818341101CC05E
:1031A0009C9CF0019D9CF00D1124EE55FD4F138267
:1031B0001282809118019601280F311D9C9CF0010C
:1031C0009D9CF00D1124EE55FD4F4281618180815F
:1031D0000E9495088394C7CF9C9C80019D9C100DF4
:1031E00011240E551D4FF80183818115F1F0815096
:1031F0008383589EC0011124648170E00E941A33B9
:10320000FB01FF27E15DFB4F8491E82FE7195E9EEC
:10321000C0011124B7010E941A3380913B04689FBA
:10322000B0011124F8017283C4CF0E94E733B501C5
:103230000E942E338C179D070CF0BBCFF3E06F1666
:1032400098F00E94E733B5010E942E33F801808385
:103250000E94E73320913A042695622F70E00E9485
:103260002E33280FF80121839C9CF0019D9CF00DCA
:103270001124EE55FD4F128280913B04893C58F099
:1032800088EC9C9CF0019D9CF00D1124EE55FD4FA7
:10329000848383838ECF8431A0F784E1F2CF0F93B0
:1032A000CF93DF93C8E3D4E0488159816A817B8161
:1032B00088E090E00E946B34288139814A815B81EB
:1032C0006C817D818E819F8100E20E948533622F17
:1032D00083E290E00E945934DF91CF910F910895DD
:1032E000E8E3F4E08DE2808311828FEF82838383B1
:1032F0001482E5E3F4E082818360828388E394E0D2
:10330000CECF80913C04833018F48F5F80933C04CF
:1033100088E394E0C4CF80913C04811519F081507A
:1033200080933C0488E394E0BACFA0E0B0E0EBE9FE
:10333000F9E10C94E232D82F062F142FE22E3091AF
:10334000380430FF35C0809139048D1308C0909146
:103350003A04961304C090913B04941729F090917D
:103360003704926090933704E32FE695E695AE2FED
:10337000B0E0A856BE4F9C91909335043C7F34300A
:10338000E1F46D2F702F812F0E940E08962F672F6A
:10339000482F892F0E94D9088D2F809339040093DC
:1033A0003A0410933B04E11419F088E394E077DFCA
:1033B000CDB7DEB7E7E00C94FE32923019F41091ED
:1033C0003B04EACF963049F3993039F3993121F72C
:1033D000E9518E2F8170D82EE695F0E0E15DFA4F2D
:1033E000C491F12C60911A01F61618F00E94BB08E6
:1033F000D3CFFC9EC001112470E00E941A338D2FA0
:10340000D1100CC0860F209118012F0D3327331FC8
:10341000412F602F0E949508F394E4CF861BF3CFD1
:10342000E8E3F4E0818121E043816281885F7DCF20
:10343000E8E3F4E0818121E043816281885075CF27
:10344000E8E3F4E0628121E1620F08F46FEF21E02C
:10345000438181816ACFE8E3F4E0628121E1621B6C
:1034600008F460E021E0438181815FCFE8E3F4E08C
:10347000438121E1420F08F44FEF21E06281818115
:1034800054CFE8E3F4E0438121E1421B08F440E03B
:1034900021E06281818149CF60913804669566950B
:1034A00070E04BE050E087E091E00E94FE33892B12
:1034B00019F481E0809336040E94110D9093260345
:1034C00080932503809137048460809337040895A6
:1034D0009091380490FF31C0811581F18B3280F5D5
:1034E0008F73880F880F909138049370892B809385
:1034F000380480913704816080933704611519F096
:1035000088E394E0CCDE609138046695669570E0BF
:103510004BE050E087E091E00E94FE33892B91F070
:103520000E943A0981E08093280320E040913B0407
:1035300060913A0480913904F8CE089581E0D1CFAA
:103540008AE2CFCFA9DFEECF8091380486958695A9
:103550008F5F8B3208F081E061E0BACF8091380450
:10356000869586958A9509F48AE261E0B1CFA9E053
:10357000B0E0EDEBFAE10C94D7328C01DC0114964B
:103580008C91811509F4BFC061E0C80161DC7C0148
:1035900080913004811136C0F8018581811509F4CC
:1035A00068C0E114F0E5FF0608F04DC0E11420E228
:1035B000F20608F0ACC0E11437E0F30619F1F0F4BC
:1035C000C701805E91090897E8F03091420480912C
:1035D00046042091410499E0F801ACE1B4E0019087
:1035E0000D929A95E1F7F0922404E0922304109250
:1035F0002604832B822B80931B0404C0E1145FE01C
:10360000F50619F7F8014581411183C133E7E31647
:103610003CE7F30609F467C0A2EAEA16A2E5FA0657
:1036200009F48FC208F064C2C7019052811590421C
:1036300008F479C2B1EEEB16F10409F482C2E5EEAA
:10364000EE16F10459C290EEE91692E5F90650F42F
:10365000A0E6EA16A2E5FA06A8F6C701925580345C
:103660009105B2CF970127573C472530310508F027
:10367000ACCFF9E7EF16FCE7FF0609F04CC020914C
:10368000230430912404232B71F1811599F081E0FA
:103690000E942C0C80911B048FD889E0ECE1F4E0AF
:1036A000A2EDB3E001900D928A95E1F78091260496
:1036B0008093D10386E0F801A2EDB3E001900D9272
:1036C0008A95E1F78091D1038093300482ED93E0F5
:1036D0004EDF10923004D80115968C91811103C0F1
:1036E00080911B0472D8809147048770811559F02E
:1036F000F8018581811539F08091A00482FF03C013
:1037000082E00E94D1052996E2E10C94F332F8019F
:103710008681803159CFBAE7EB16BCE7FB0609F08A
:1037200071CF811509F4CAC0A0902304B09024047D
:10373000E0911B04E887E983BE016F5F7F4FC501FD
:103740000E94440B2C01F981F987FBEDCF2EF3E0A9
:10375000DF2EEE24E394F12C22242A94D60117962E
:103760003C90179733FE54C06D907C901197129641
:103770008D909C90139746145704B9F41496BC91FD
:10378000BF83232DF60146816B2F89850E945E0B36
:10379000811559F08F810E94E804281634F4D6016F
:1037A00015969C917401F92A282E48145904C9F4DD
:1037B00031FE17C0F601F581FF83232DD601169641
:1037C0004C916F2F89850E945E0B811551F08F817E
:1037D0000E94E80428162CF4F60194817301F92A5A
:1037E000282E30FE15C0FFEF2F1212C021E0E21686
:1037F000F10471F4232DD60116964C9160E0898571
:103800000E945E0B811521F0F60185817401F82A72
:10381000F8E0CF0ED11C2BE134E02C153D0509F06A
:103820009DCF31E0E316F104F1F5988592959F70F4
:103830004885942B9F7081E0403108F480E0F82E99
:10384000F294E0EFFE22F92AA11450E2B50620F529
:10385000A11481E0B80608F055C0EA2C8F2D8D70B8
:103860004A2D811509F451C06AE08BEF98E00E945F
:103870003D0C282F30E02115310551F44E2D66E125
:103880008DED98E00E943D0C282F30E0811549F025
:10389000F901FF297F0107C0C501905281159043AE
:1038A00090F1E12CF12C87E0E7E2F4E0DF011D92DA
:1038B0008A95E9F7F0922F04E0922E0480912E046D
:1038C00090912F04892B09F40ECFF8018581811581
:1038D00039F08FEF0E942C0C8091260480932504F0
:1038E00086E0F801A7E2B4E001900D928A95E1F735
:1038F000809125048093300487E294E038DE1092B2
:103900003004F1CEFB28BB24A8CF68E083EF98E019
:10391000AECFC70197578038910508F0D3C5BE2CAC
:10392000F0E1EF1608F0DFCE66EB70E080E090E0AB
:10393000F0DA8111D8CEC12CD12C7601B11045C05E
:1039400074E0272EAE014F5F5F4F5E834D83AD81E4
:10395000BE81E22D1D92EA95E9F746015701FFEF7E
:103960008F1A9F0AAF0ABF0AC701B601D2DA89834C
:10397000811509F4B8CE813009F0A5C026013701C0
:1039800022E0420E511C611C711CC501B401C1DA58
:10399000382E8A83811509F4A6CE8FEF830D8330EC
:1039A00038F5C301B201B5DA8B83811521F0CE0160
:1039B00001960E94F8134601570133E0830E911CD3
:1039C000A11CB11C75016401C2CF27EBC216D10442
:1039D000E104F10409F487CEC701B6019ADA3FEF9A
:1039E000C31AD30AE30AF30A8111EFCFBA94A6CF20
:1039F0008BEF830D833090F54601570143E0840E31
:103A0000911CA11CB11CC301B20183DA8B83811507
:103A1000C9F2C501B4017DDA8C83811108C0460169
:103A2000570154E0850E911CA11CB11CCBCFAB807B
:103A3000BC8081E0A8168FEFB80610F0BA2CAA243B
:103A400096E0391641F0A7E03A1611F0C501A5D766
:103A5000C501D5D7E4CFC501A0D7E1CFB4E053016C
:103A600042013B12AFCFC301B20153DA782E4601B7
:103A70005701E4E08E0E911CA11CB11CC701B601D8
:103A80006D5F7F4F8F4F9F4F44DA711409F42BCE37
:103A9000811509F428CE8150990B4FEF489F900172
:103AA000499F300D1124472D4150550B240F351FD0
:103AB0002150310908F486CF8FE99FE00197F1F793
:103AC00000C00000F5CFCE0101960E94F8137ACF16
:103AD000109242040E94F4050E94B80C88579C4E34
:103AE000909333048093320481E080933104FBCDC2
:103AF000F2EBEF16F2E5FF06E9F525EE30E0277070
:103B0000332781E090E001C0880F2A95EAF72091E1
:103B10003404309131043115E1F04115A9F0282B1E
:103B200020933404E0CDD80116968C91803110F5A5
:103B30008F2D99278F7199278230910511F0429727
:103B4000DBCF21EE30E0DBCF8095822380933404FD
:103B5000CACD322F3823311569F0982F90959223D2
:103B6000909334040E94EC05D80115968C91811530
:103B700009F4B9CD80913104811509F46DC0C0906C
:103B80004204D09041040E94B80C88579C4E9093F8
:103B9000330480933204F8018581811509F45CC0F7
:103BA0008D2D8C298D79811182C0E114F0E5FF06FD
:103BB00008F5E11420E4F20608F083C036EEE316BF
:103BC000F10409F449C0C70190528115904208F0F0
:103BD0007FC0D80116968C91803108F460C0C7016F
:103BE0009927109246048D32910509F582E0809361
:103BF000460472C0B0EEEB16B2E5FB0608F03FC01B
:103C0000E0ECEE16E2E5FE0638F5F0EAEF16F2E536
:103C1000FF06E8F420E6E21622E5F206E8F4C70122
:103C2000925580349105C0F010924604C7018E323F
:103C3000910508F05EC08832910508F04BC08E31C6
:103C4000910508F049C004974A9780F230C034EBE0
:103C5000E31632E5F30641F7F8019581911509F471
:103C600027C4809142048272F701E052F847EB309A
:103C7000F10508F088C0E950FB4C0C94413349E74A
:103C8000E4164CE7F40630F457E7E5165CE7F50672
:103C900018F7CACF8BE7E8168CE7F806DCCF8F2D34
:103CA0008F718431C9F2863111F4109246040E945A
:103CB000EF138091420490913404892B8093420445
:103CC000CBCFD80116968C91803108F088CFC4CF25
:103CD000C70187CF8A9759F780913404811531F055
:103CE0008091460492E08927809346040E94EB0F5E
:103CF000B3CF8C34910581F38D329240ECCF80911B
:103D0000380480FF10C08E7F8093380488E394E0ED
:103D1000C6DA0E943A0980913704816080933704A3
:103D20000E94BB08E0CC81608093380461E08695F6
:103D30008695CEDBD8CC811521F010DCD4CC811552
:103D4000E1F302DCD0CC811521F072DBCCCC811503
:103D5000E1F366DBC8CC811521F07DDBC4CC811595
:103D6000E1F36EDBC0CC811521F08BDBBCCC81157F
:103D7000E1F37CDBB8CC811521F0CDDAB4CC811530
:103D8000E1F3BFDAB0CCF7E7EF16FCE7FF0609F185
:103D900028E7E2162CE7F20629F19701205E32456A
:103DA0002032310520F5911122C03E2D3F7181E076
:103DB00090E0AC0102C0440F551F3A95E2F77A013A
:103DC000642F83E090E00E9459348E2D0E94FE04FF
:103DD0008ACC81E00E94040543E062E081E00E9419
:103DE000A80581CC82E0911509F469C3F3CF409115
:103DF000400480914504282F30E02095309570E0F4
:103E000024233723232B19F04823409340045BE7F6
:103E1000E5165CE7F50641F4911509F464CC0E94BF
:103E2000EB040E94050C5FCC80E4E81682E5F806FE
:103E300008F096C0A0E2EA16A2E5FA0608F0BFC0B4
:103E4000E114B0E5FB0608F066C0E114E0E4FE060C
:103E500008F0CBC0D80117968D919C91009709F47A
:103E6000FEC00E94F206D82EF92ED8011596BC90FD
:103E700015971696AC90A2942FE0A2228091470449
:103E80008770811509F1CB2CB114F9F0892F807F4F
:103E9000803469F080E28D0D8830B0F0892F807E0B
:103EA000803229F4B2E0DB1678F0A11469F0809139
:103EB000A00482FF09C082E00E94D10580914704DE
:103EC0008770CC24C3948111C12C8F2D82958F7063
:103ED000883009F4E7C108F0F6C0843008F0D7C094
:103EE000EF2DEF70EE2E823008F4FEC08F2D807F14
:103EF000803219F0E29480EFE822D11409F42CC149
:103F000031E0D31609F490C1B11409F49CC1A11495
:103F100009F440C100C1970130552115324008F025
:103F200099CF970145E0369527954A95E1F7822F7D
:103F30008F702091400430E041E050E0082E02C034
:103F4000440F551F0A94E2F724233523232B09F449
:103F500081CF911166CF109242040E94EB0FC3CB28
:103F60009701205C32452032310548F1911509F462
:103F700071CFBAE5EB16BCE7FB0609F46CC008F09C
:103F80004EC0F1E0EF16FCE7FF0609F462C023E043
:103F9000E2162CE7F20609F456C0E1143CE7F306FA
:103FA00009F058CF0E943A108FEF94E3ACE08150B3
:103FB0009040A040E1F700C000000E94C00E8E2D8E
:103FC0008F712091400430E041E050E0082E02C0A3
:103FD000440F551F0A94E2F724233523232B09F4B9
:103FE00039CF911509F47FCB1CCFD80116968C914F
:103FF000803108F02FCF91112DCF2F2D2F7081E020
:1040000090E002C0880F991F2A95E2F720914004A2
:1040100030E082239323892B09F41CCF64CB4BE53A
:10402000E4164CE7F406C9F08091A004002482FF56
:104030000394802D5CE5E5165CE7F50609F00ACFF0
:104040000E947B0F07CF6FEF7FEF80E090E00E9430
:1040500073340E944C1081E0F3CF80E0F1CFF8017F
:104060008581C080D180811569F0C6010E94FE164D
:10407000F82E682FC6010E947205B6018F2D0E948E
:10408000D416EFCEC6010E948D05F82EF6CF8430EF
:1040900009F4EBC0C11409F435C18091470480FDD7
:1040A00031C1D80115961C928695869586950E94F9
:1040B0000405C8015CDA809147048695869586954B
:1040C0000E940E051FC1893009F461C18A5F8F709B
:1040D000823000F7F2EFDF126DC18F2D8F71B110BA
:1040E00066C10E9404050CC120E1F21618F0E294AA
:1040F00090EFE922B114B9F0E11469F080E28D0D7E
:10410000883010F0D11009C0809142048E2980932C
:1041100042040E94EB0F8D2D2FC0809146048E2902
:1041200080934604F6CF8D2D0E948913E11409F483
:10413000B1CF80E28D0D883010F0D11004C08E2DEB
:104140000E94EC0506C0E094809146048E21809385
:1041500046040E94EB0F9ECF8091A00482FD16C002
:10416000B11469F0E11439F0809142048E298093F2
:1041700042040E94EB0F80E00E9424138BCF80E06A
:104180000E948913E11409F485CFD9CFB11471F1DC
:10419000A11004C08E2D0E94CD137CCF41E0A4124B
:1041A00011C0F09041048E2D8F21E81609F472CFD2
:1041B0000E94B80C90934B0480934A04FE28F0921E
:1041C000410468CF55E0A51265CF8E2D0E94CD1316
:1041D0008E2D0E94D80C809143049E2D9823E916C1
:1041E00009F458CF8E298093430454CFA11012C0F4
:1041F0008E2D0E94D6138E2D0E94D80C80914304E0
:104200009E2D9823911509F445CFE094E822E09281
:10421000430440CF81E0A8123DCF809142048E211B
:10422000811509F437CFE4CFB11429F096E0A9162F
:1042300008F030CFAFCFA5E0AA1608F02BCF8E2D17
:104240000E94D61327CFA114D1F3B9E3DB1209C022
:10425000EFEFF7EE23E0E150F0402040E1F700C03F
:1042600000008D2D0E94891315CF8F2D8695869580
:104270008370811569F0813009F00CCF8D2D9F2D51
:104280009370B11002C080E090E00E948D0C02CFCC
:104290008D2D9F2D9370B11002C080E090E00E94A0
:1042A000650CF8CE8F2D8370811139C0B11028C0F4
:1042B0004D2D429546954770440F440F8D2D8F70BC
:1042C000042E01C0880F0A94EAF72D2D2071D4FE28
:1042D00007C02FE030E001C0220F4A95EAF7209591
:1042E0003F2D3695369533703230A1F0333081F062
:1042F00040914404313059F0822B84230E94FE0403
:104300000E94520C60E0C8010E942817FCC9842B4F
:10431000822BF4CF822B909144048927EFCFB114E4
:1043200059F1F0FEEDCF4D2D429546954770440F63
:10433000440F8D2D8F70042E01C0880F0A94EAF768
:104340002D2D2071D4FE07C02FE030E001C0220FD8
:104350004A95EAF720953F2D3695369533703230E1
:1043600089F0333069F040914504313041F0822BBF
:1043700084230E940105C4CF8230A8F6C1CF842BCC
:10438000822BF7CF822B909145048927F2CF3F2DC6
:104390003F70F32EB11439F0832F0E9404058D2D48
:1043A0000E94CD13ADCF8D2D0E94D6138F2D0E946C
:1043B0000E05A6CF43EFD41680F450EFD516E1F0EA
:1043C00081EFD816A1F0B11409F460C0A11409F46A
:1043D0005AC08D2D0E94241393CF93EFD916F1F07C
:1043E000A4EFDA12F0CF8091A00482FD23C08F2DBC
:1043F0008F71B114E1F275CEB11469F0B5E0AB166E
:1044000008F07ECF2F2D2F7181E090E001C0880F42
:104410002A95EAF7B8CFE6E0AE16F2CF80E0B11405
:1044200009F4A7CF9F2D9F7181E001C0880F9A9555
:10443000EAF79FCFB114C1F08091470487708430B0
:1044400049F41092470410924904109248048F2DA9
:104450008F71ADCFF5E063E0AF1608F051CF8F2D2F
:104460008F710E94C40C4CCF25E0A21640F0109230
:104470004704109249041092480464E0F0CF81E0B0
:104480000E94D1053DCF8F2D8F712BCEA114F9F253
:1044900039E3D31209C04FEF57EE83E0415050404B
:1044A0008040E1F700C000008D2D0E94891328CFC5
:1044B000F7E7EF16FCE7FF0609F06ACC81E00E94FF
:1044C0000E058ACC23E7E2162CE7F20609F0A4C811
:1044D00080913104811509F4FBCA0E94EF1303C9CE
:1044E00080919C04803178F480919B04811559F06F
:1044F000E0914D0420914C04309197044091960432
:1045000059E02E1301C008956E2F70E05E9FF001F8
:104510001124DF01A25BBB4F14968C911497811577
:1045200059F111968C911197831326C08C918413A5
:1045300023C015968C91159781111EC012968D91EE
:104540009C91A0919804B09199048A1B9B0B883C84
:10455000910590F480919C048F70806180939C04FD
:10456000EC5AFB4F80818F708061808386E994E0F4
:104570000E94B71A0C94C705FB013196E770C1CFB2
:10458000AFE0B0E0E6ECF2E20C94DB328C0186E0C6
:10459000F801DE011A9601900D928A95E1F7F80173
:1045A000F580848196E9892E94E0992E60909A0492
:1045B000611017C0811591F0F11409F417C1C801F9
:1045C0000E945717811509F411C189E0F801A6E985
:1045D000B4E001900D928A95E1F782DFFF24F39415
:1045E00056C07080A280B380D0909B042091980424
:1045F00030919904A501421B530BD11409F4C6C094
:10460000483C510508F079C0811541F38091970429
:10461000C180E0909C0450E1E51608F059C0C81232
:1046200015C080919604871111C0F1104BC08E2DDA
:104630008F70806180939C0486E994E00E94B71A91
:1046400080919C04F8018683F12C21C0F1103AC0BE
:1046500040E06C2D872D0E947B0E40E06C2D872D55
:104660000E947B0EF82E8111EFCF8A859B850E94D8
:104670004A17292F22952F70903470F49F702230A2
:10468000A0F09115B1F0F8019681903190F48F2D42
:104690002F96EEE00C94F7322A5F2F70223068F0EC
:1046A000C8010E94B71AFD2CF2CF911511F08115A7
:1046B00071F3805E883058F3F3CF803F40F3815F21
:1046C0008330F9CF80919C04816080939C04BCCF9F
:1046D000C8123BC080919604871137C0F11035C0D5
:1046E000E682C8010E94B71A89E0F801A6E9B4E0A1
:1046F00001900D928A95E1F771CFE0909C04F0E172
:10470000EF1650F486E994E00E94B71A89E0F401AC
:1047100011928A95E9F798CF811509F45FCF9091AE
:104720009704F8018181981310C080919604871135
:104730000CC0F1100AC0E682C8010E94B71A89E0D5
:10474000F40111928A95E9F749CFC8010E945717E1
:10475000811509F44BC0F11409F448C080919C0400
:10476000803208F432CF1E821F821886198680910B
:104770009604909197049A838983BC82AB826D8260
:10478000EF82CE0101960E94B71A1FCF483C510517
:1047900008F0BCCF811509F421CFF11439F19091C3
:1047A00097048181981318C080919604871114C0D2
:1047B00080919C0480FD98CF803108F495CF86834A
:1047C000807F803F09F48DCF8681982F907F905F06
:1047D0008F70892B868385CFC8010E94571781115E
:1047E000F4CE80919C04816080939C04C8010E9457
:1047F000B71AF4CEA1E2B0E0E0E0F4E20C94E532C6
:104800004C8F5D8F6E8F7F8F88A3192F99A3911185
:1048100010924604198E1A8E1B8E86E0FE017C963D
:10482000DE01539601900D928A95E1F708A18091DF
:10483000A00482FF1FC00E94B80C20914804309150
:104840004904821B930B8838934138F080914704C8
:1048500082FD03C082E00E94D1050E94B80C209125
:104860004A0430914B04821B930B8838934110F01B
:104870000E94F405011561F00F8B188F61E0CE01E5
:1048800043960E94281761E0CE0143960E942817A4
:104890000F8B188F89E0FE017396DE011A96019046
:1048A0000D928A95E1F7CE010A966ADE811110C059
:1048B00020914C0430914D0489E0FE013A96DE01CE
:1048C000119601900D928A95E1F78E8581110BC0AA
:1048D00019E080914D0490914C0489132BC0A1964E
:1048E000E4E00C940133822F90E0019687709927C1
:1048F0003817190671F40E943A1010924C04109265
:104900004D0489E0E6E9F4E0DF011D928A95E9F7BC
:10491000DFCF99E0929FD0011124A25BBB4FFE0133
:10492000319601900D929A95E1F780934C040E9484
:10493000C705CECF189FC0011124825B9B4F20DE9C
:10494000811569F280914D0490E001968770992756
:1049500080934D04BECFA6E0B0E0E1EBF4E20C940E
:10496000E5320E94B80C8C0180919E0390919F03C8
:104970008017910771F019821A820E94B80CBC014D
:1049800049815A8180E090E035DF10939F030093C6
:104990009E032696E4E00C940133A6E0B0E0E3ED3C
:1049A000F4E20C94E5328C0190939B0380939A037C
:1049B000011580E21807B0F4C801805E91090897DC
:1049C00028F06CED73E10115110511F46DEC73E144
:1049D000C8010E94BC04802F0E9424132696E4E0A4
:1049E0000C94013380EF89838A830E94B80C816024
:1049F000BC0149815A8181E091E0FCDEEFCFA6E065
:104A0000B0E0E5E0F5E20C94E5328C0190939B0375
:104A100080939A03011580E21807B0F4802F0E945A
:104A20008913C801805E9109089728F065EE73E14B
:104A30000115110511F466ED73E1C8010E94BC0473
:104A40002696E4E00C94013380EF89838A830E94E8
:104A5000B80C8160BC0149815A8181E090E0CADED6
:104A6000EFCFACE0B0E0E7E3F5E20C94E13280E0B8
:104A70001CEF0DEFFF24F39490912E0320912D0352
:104A8000291709F441C0E92FF0E0E15DFC4F808176
:104A900087FBCC24C0F8D82EE894D7F89F5F93709A
:104AA00090932E0390912C039F5F90932C0387FD8E
:104AB00007C0DF8218870E94B80C23E0E22E06C0F0
:104AC000DF8208870E94B80C32E0E32EBC018987A0
:104AD0009A87EB86FC864F8158858E2D91E08ADE81
:104AE000D982C11479F00A830E94B80CBC018B836F
:104AF0009C83ED821E8249815A818E2D90E07ADE60
:104B000081E0BACF1A83F0CF2C96E8E00C94FD3206
:104B1000AFE1B0E0EEE8F5E20C94D932FE01319657
:104B200084E1DF011D928A95E9F766E2E62E61E0F5
:104B3000F62E8F017BE2672E71E0772E2F01AA24DB
:104B4000A394B12CF6E28F2EF1E09F2EF701819114
:104B50007F018F3F09F444C0F894E82FE295EF708D
:104B6000F0E021A18F70A50102C0440F551F8A9566
:104B7000E2F7CA01922F982B91A392A180958923E5
:104B800082A3789400C0EDE1F1E021E030E0C12C97
:104B9000D12C41914F3F79F0A42FA295AF70A05E28
:104BA000B0E08C9190E04F7002C0959587954A9542
:104BB000E2F780FF8FC080E090E0C82AD92A220F58
:104BC000331F8E169F0629F7F70182918F3F11F050
:104BD0000E94F00750EA5A95F1F7D801CD92DC9285
:104BE0000E5F1F4F6E147F0409F0B0CF44E150E018
:104BF000B20184EF92E00E940B349C01892B41F0BA
:104C000084E1F201A4EFB2E001900D928A95E1F700
:104C10000091090310E0000F111F025C1C4F232BB1
:104C200009F45AC081E0809355020E94B80C909319
:104C300054028093530280919803811509F4A8C00F
:104C40007E01B5E1EB0EF11C8AE0F70111928A9525
:104C5000E9F7809156028A3008F062C047E255E1D8
:104C6000B701C8010E94410F811509F47FC042E5D8
:104C700055E1B701C8010E94410F811509F476C0C2
:104C80004EE955E1B701C8010E94410F811509F4B1
:104C90006DC049EF55E1B701C8010E94410F811570
:104CA00009F464C0109256028091080390E0880FC6
:104CB000991F4AE050E0B701825C9C4F0E940B3480
:104CC00021E020935202892B09F041C06F96E0E168
:104CD0000C94F532C90171CF80915502811509F408
:104CE000AACFE0905302F09054020E94B80C8E19A3
:104CF0009F09059708F49FCF4AE050E064EF72E007
:104D0000C8010E940B34892B41F08AE0E4EFF2E005
:104D1000D80101900D928A95E1F7109255028BCF40
:104D2000C0905002D09051020E94B80C8C199D097D
:104D3000843F914008F092CF80915202811531F268
:104D40008AE0D7011D928A95E9F710925202A0914C
:104D50000803B0E0AA0FBB1FA25CBC4F8AE0FE01B3
:104D6000759601900D928A95E1F7B0CF8091560229
:104D70008F3F39F40E94B80C9093510280935002F7
:104D8000DBCF8F5F809356028A3008F48DCFF2CF4D
:104D90008AE0F801A2E7B3E001900D928A95E1F76D
:104DA0006AE070E082E793E00E94ED0B809371036C
:104DB00088E0EBE2F3E0ADE7B3E001900D928A9575
:104DC000E1F768E070E08DE793E00E94ED0B8093DF
:104DD0007C03C0908503D0908603E0908703F09019
:104DE000880380914C0290914D02A0914E02B091A7
:104DF0004F02C816D906EA06FB06B1F0C0924C0273
:104E0000D0924D02E0924E02F0924F020E94ED0CC1
:104E1000C61AD70AE80AF90AC0929403D0929503F9
:104E2000E0929603F09297038BE0E9E8F3E0DE016D
:104E3000559601900D928A95E1F7F0908A03E090E3
:104E40008B03D0908C0300919203109193031092E6
:104E50009303111509F43ACF10FF0DC08D8980FF1F
:104E60001EC09091380491609093380460E086955C
:104E700086950E94681A11FF06C020E04D2D6E2D08
:104E80008F2D0E94951912FF04C0011559F00E9440
:104E90004C1A13FF1BCF81E08093280317CF0E9489
:104EA0004109E9CF0E943A09F4CFA0E1B0E0EBE577
:104EB000F7E20C94D932FE01319680E1DF011D92B8
:104EC0008A95E9F70CE010E099E4A92E93E0B92E59
:104ED00027EB422E512C612C712C4F017301620182
:104EE000B1E14B165104610471041CF080E1C82E3D
:104EF000D12CA601B501C4010E944A34AC0CBD1CE2
:104F00000D2C000CEE08FF084C185D086E087F0899
:104F10000150104019F76096E0E10C94F5326FEF04
:104F200085E290E00E9459346FEF86E290E00E94A3
:104F300059346FEF87E290E00E94593460E088E2D4
:104F400090E00E9459340E94F217AFDF67ED85E2CE
:104F500090E00E9459346EE786E290E00E94593456
:104F60006DE287E290E00C9459348F929F92AF9259
:104F7000BF92CF92DF92EF92FF920F93CF93DF9386
:104F800088E090E00E9440344B015C01C8E3D4E02B
:104F900068839982AA82BB821C821D821E821F8224
:104FA00083E290E00E943834282F30E040E050E067
:104FB00060E070E080E090E000E20E946A3328291F
:104FC00039294A295B29288339834A835B836C8387
:104FD0007D838E839F83DF91CF910F91FF90EF9020
:104FE000DF90CF90BF90AF909F908F900895CDB7F6
:104FF000DEB7AA970FB6F894DEBF0FBECDBF85B758
:10500000806885BF85B7806885BF84B7877F84BF88
:105010000FB6F894A8958091600088618093600035
:10502000109260000FBE80E890E00FB6F894809375
:105030006100909361000FBE81E0809315018EEEB8
:1050400097E090934302809342020E94B2170E941D
:10505000C40D0E94210E8091E20084608093E200E2
:10506000789480915403811599F08091E900109112
:10507000EC008F70179511271795182B1092E900E7
:105080008091E80083FD0E9461101F701093E90079
:1050900082E084BD93E095BD9AEF97BD80936E004A
:1050A0001092940310929503109296031092970316
:1050B0000E949917811101C032DF8091D800806170
:1050C0008093D8002AE12A95F1F700C08091D90099
:1050D000182F117080FD04C00E94C40D109254035B
:1050E0001093980387988F988FE891E00197F1F7D4
:1050F00000C000008FB187FB992790F99093990326
:1051000090932B018038880B8195880F880F880F2A
:105110008093160188E08093170180919803811194
:105120000E948431EBE2F3E088E0DF011D928A9572
:10513000E9F780912B0191E08927809335038091D5
:105140002B019093380380912B0180912B018111C9
:1051500006C086E980931C0184E980931B0160E00E
:1051600080E00E94A00B61E080E00E94A00BEFE8CD
:10517000F1E03197F1F700C0000010E080913803B2
:10518000181708F4BCC080912B01811124C085E060
:10519000E0E7F1E0DE01919601900D928A95E1F74A
:1051A00085E0FE01B196A6E2B1E001900D928A95EC
:1051B000E1F789E0E6E7F1E0DE01119601900D925A
:1051C0008A95E1F789E0FE013196ADE1B1E0019009
:1051D0000D928A95E1F780912B0190E0811101C039
:1051E00095E09093090385E0891B8093080306E20C
:1051F00011E09BE2E92E91E0F92ED8018D918D010D
:105200008F3F11F00E94F007E016F106B1F70DE1B3
:1052100011E086E2E82E81E0F82EF80181918F01FD
:105220008F3F11F00E94F007E016F106B1F784E11C
:10523000EEE3F3E0DF01282F1D922A95E9F7E4EF72
:10524000F2E0DF011D928A95E9F780E090E00E948C
:105250004534833E9E4F21F40E94991781112AC044
:1052600063EE7EEF80E090E00E94733460E082E0C5
:1052700090E00E94593481E08093440461E083E02F
:1052800090E00E94593460E074E184E090E00E9474
:1052900073340E94701943DE40E050E0BA018FE0A1
:1052A00090E00E946B3440E050E0BA0183E190E06E
:1052B0000E946B3482E090E00E94383480930D03AA
:1052C00084E090E00E9445349093A00480939F0472
:1052D0001FDCEFEFF6E721E0E150F0402040E1F77E
:1052E00000C0000015DC80913E0380FF1AC06FEF04
:1052F0007FEF80E090E00E9473340E94C00E60E077
:10530000812F0E94C30B082F61E0812F0E94C30BE5
:10531000E12FF0E0EA5CFC4F880F802B80831F5F59
:105320002DCF83E090E00E9438340E94FE048091EB
:105330000A03811123C088E394E017DE80913704CB
:1053400083608093370480913804843028F40E946D
:10535000701988E394E009DE0E94AD080E943A09C2
:105360000E94E00B8091380480FF05C060E08695C4
:1053700086950E94681A81E080930A0380919803C1
:10538000811101C0C4D78CE291E09093A103809376
:10539000A0038091540310E402E1853009F48EC02B
:1053A000B7DB1EE0812E13E0912E0EE3402E03E0CA
:1053B000502ED201F401219131918D919D9143E0C4
:1053C000E232F40709F484C028173907A1F33090BA
:1053D0009803BEE36B2EB3E07B2E10E0D301ED907B
:1053E000FD903D01F401A190B1904F01AE14BF04B6
:1053F00059F1AE24BF2400E0CC24C394D12CC601C3
:105400008A219B21892BC1F03114B1F009831A83C1
:105410000E94B80C9C838B83F1E0FD8391E09601A0
:105420002E213F21232B09F490E09E8349815A814C
:105430006B817C818D81DED90F5FCC0CDD1C093046
:10544000F1F6F401F292E2921F5F1A3039F60E94EF
:10545000F90C43C080915403843019F110920B036E
:1054600048E150E00FB6F894A895409360000FBE55
:105470001093600083B7817F846083BF83B78160AE
:1054800083BF7894889583B78E7F83BF0FB6F894D7
:10549000A895809160008861809360001092600000
:1054A0000FBE36DBEEE3F3E081919191892B09F099
:1054B0003EC582E593E08E179F07B1F780915403B4
:1054C000853009F4C7CF0E943A100E94520C68CF71
:1054D0002817390709F07BCF3EDA809198038115B0
:1054E00089F080913104811569F00E94B80C2091F7
:1054F000320430913304821B930B8F3F9F4710F48B
:105500000E94EF1380913604811509F46FC08091D9
:105510003504E0913804E695E695E81BE09327030F
:10552000853109F4CEC008F084C0893009F4BFC0C9
:1055300008F072C0823009F4A8C0863009F4AEC009
:10554000E0EDEE2EE7E0FE2E0DE018E0809128035E
:10555000811561F0109228030E94110D909326038B
:105560008093250310922A03109229030E94110DA3
:105570009C018091250390912603A901481B590B9A
:105580004F3F5F4798F5409124034115B1F01092C9
:1055900024034091220350912303241B350B2F3FFA
:1055A0003F4758F4405D5A485093230340932203E9
:1055B00020913704286020933704A0902903B090ED
:1055C0002A038E0D9F1D909326038093250385E269
:1055D00093E0F80109958091290390912A03892B82
:1055E00029F4AB2819F0F1E0F0932403D09098034C
:1055F000D11411F036DAD82E80915D03811551F067
:1056000010925D0380912D0380932E0380912B03D4
:1056100080932C03C12C99C08F3009F091CFE6956F
:10562000F0E0E45BF94FE491EE2EF12C02E919E091
:105630008DCF74EFE72EFF24F39402E11BE0843258
:1056400009F484CF90F468E2E62EF12C00E91AE028
:10565000883109F47BCF833209F072CFE7E4F6E0BA
:10566000E590F59000E019E071CF853209F068CF40
:105670008E2F63E0D3D7E92FF0E0EC5BF94FE49194
:10568000EE2EF12C0EE818E161CFF0E0EB5AF94F65
:10569000E491EE2EF12C0DE419E058CFF0E0EE5A33
:1056A000F94FE491EE2EF12C0BE219E04FCFE69585
:1056B000F0E0E15BF94FE491EE2EF12C00E619E009
:1056C00045CFF0E0E75BF94FE491EE2EF12C01E1DC
:1056D0001AE03CCF61E08C2D0E94C30BF82E60E0F5
:1056E0008C2D0E94C30BFF0C8F292C2D30E0D9018B
:1056F000AA5CBC4FEC919E2F9370891729F1EE0F95
:10570000EE0FE82BEC93809135038C0DEF70F0E0F9
:10571000ED53FE4FA9014D5C5C4F7A01B080DA0178
:105720009C91B90EB4E060E0BB1624F4EDEFBE1618
:105730001CF461E00E947F0B8B2DBB0C990B64E085
:1057400070E08CD7D7018C93C39480913803C8162E
:1057500008F4C0CF80919803811511F082D9D82A1E
:10576000D1100E94F90C0E94520C909139038917B4
:1057700021F0809339030E94ED0C80915403843012
:1057800009F007CE83E08093E9008091E80082FF72
:1057900000CE8091E80090E085FF05C00E94930D47
:1057A000811529F191E08091E8008B778093E800E2
:1057B000911509F4EECDE0909C03F0909D03E981F2
:1057C000E114F10491F1EE3F09F051C08A81833078
:1057D00020F08550833008F04AC0EA81EE3008F0AE
:1057E00046C0F0E0EE5FFA4CCE0101964AC750E2A7
:1057F000E52EF12CFE0131966F018091E80085FDC8
:105800000AC08091E8008B778093E8000E94930D96
:10581000811599F3C7CF8091F100D6018D936D0169
:10582000B1E0EB1AF10849F7BDCFE43148F4E115D6
:1058300049F0E150E33130F4F0E0E05FFA4C21C789
:10584000EE3F59F28FEF898312C01A8289E08B8371
:105850000EC08A81823081F08330B1F0813091F7BF
:105860000E94ED0C24D76B837C838D839E83CE01B5
:1058700001960E94E30D8DCD88E290E0F9D71B825E
:105880001C821D828E83F3CF80915203909153032B
:10589000892B69F3FE01319682E593E0D2012C91C8
:1058A00011963C91B2E04B0E511C32832383329609
:1058B0008415950599F7DBCF8A81823019F66B81C3
:1058C0007C818D819E81F3D688E290E0F2D7CFCFA4
:1058D0004C816B818A810E946C16982789279827B2
:1058E0009E838D83C4CF2D813E813227232732278B
:1058F0004C816B818A810E94920FB9CF0E94F2176E
:10590000B6CF8A81823869F178F48038B1F0813875
:1059100009F0ADCF60E08B810E94681A8B81811104
:1059200015C00E944109A3CF833809F0A0CF20E021
:1059300040913B046C818B8106C020E04B816091DB
:105940003A04809139040E94951991CF80913804CE
:1059500081608093380460E0869586950E94681A7D
:1059600086CF8B8180933C0482CF8A818238E1F09C
:1059700060F48038A1F0813809F079CF8091380443
:1059800080FF10C08695869562CF833809F06FCF6F
:10599000809139048B8380913A048C8368CF809105
:1059A0003B0455CF80E053CF80913C0450CF0E9400
:1059B000AD0888E394E00E944F1959CF80E18A83B3
:1059C00056CF1A8287EB43CF0C810D3108F04FCFB1
:1059D0008A809B80982489249824A12CB12CFE01D4
:1059E00031967F010E0F1F2F111D0E151F0509F493
:1059F0003ECF80E0F7EB8F169104A104B10420F4B0
:105A0000C401875B9C4F34D7D70114968C93BFEFAA
:105A1000EB1AFB0AEFEF8E1A9E0AAE0ABE0AE5CF1A
:105A20008091520390915303892B09F420CF8C81EC
:105A30008D3108F01CCF882E912CA12CB12CCA805E
:105A4000DB80DC24CD24DC24E12CF12C8E010F5FE3
:105A50001F4F412C512C3201481459046A047B0415
:105A600008F005CFF7EBCF16D104E104F10438F4C8
:105A7000D80114966C91C601875B9C4F1AD7BFEF73
:105A80004B1A5B0A6B0A7B0AEFEFCE1ADE0AEE0AAC
:105A9000FE0A0F5F1F4FE0CF08DAE9CE84E08FCF18
:105AA0008C818D3108F0E3CE882E912CA12CB12C65
:105AB000CA80DB80DC24CD24DC24E12CF12C412CB9
:105AC000512C32018E010B5F1F4F481459046A0498
:105AD0007B0408F0CCCE80E0F0EDCF16F2E0DF06DC
:105AE000E104F10418F4C6018996C2D6D8018D9359
:105AF0008D01BFEF4B1A5B0A6B0A7B0AEFEFCE1AE0
:105B0000DE0AEE0AFE0AE1CF2C81022F10E02D31D1
:105B100008F0ADCE8A819B819827892798272C0190
:105B2000612C712C803DF2E09F0708F0A0CE822E00
:105B3000912CA12CB12C40ED52E060E070E04419B2
:105B4000550966097709421751056105710508F481
:105B50008ECE2091520330915303232B09F03EC087
:105B60001C0129E2220E311C80FBEE24FF24E0F808
:105B700080FF0BC088967CD69D818927982789272E
:105B800081159C4711F48FEF8D83D501C401840DDD
:105B9000951DA61DB71D80FF19C0680141E0C41AFC
:105BA000D108CE0105968C0D9D1D9AA789A7C1012C
:105BB000800F911F5DD6A9A5BAA59C9181159C4720
:105BC00021F48FEFE9A5FAA580838601FE013196C5
:105BD000EE0DFF1D2FEFE016F10638F08E010F5F7E
:105BE0001F4FC12CD12C760125C094818581811550
:105BF0009C4711F42483258342E0E40EF11C329685
:105C0000EACF50ED451652E055066104710430F4B8
:105C1000D80114966C91C20189964BD6BFEFCB1A6E
:105C2000DB0AEB0AFB0AEFEF4E1A5E0A6E0A7E0AE7
:105C30000F5F1F4FC814D904EA04FB0410F317CEFA
:105C40008091520390915303892B09F410CECE0119
:105C500001960E94E30DFFEF21EE34E0F150204069
:105C60003040E1F700C0000048CB88E0E0E8F1E018
:105C7000DE01919601900D928A95E1F7FE01329630
:105C80008FE1DF011D928A95E9F786E0898388E03C
:105C90007F96DE01159601900D928A95E1F7E7CD8A
:105CA00084E8898382E08A831B821C82E0CD0B8199
:105CB0001C81012E000C220B330B45E0000F111F3D
:105CC000221F331F4A95D1F7B901A801405E5F4FEB
:105CD0006F4F7F4F401751076207730708F4C7CD16
:105CE0000438B2E01B072105310508F0C0CD453866
:105CF000E2E05E076105710520F044E852E060E0F3
:105D000070E0401B510BB801675A794F6ED5AFCD8B
:105D10001B810C8140E0602F812F0E949B169827E9
:105D2000892798279A83898341E0602F812F0E94D9
:105D30009B169827892798279C838B8398CD2E8143
:105D40003F812C37310569F032272327322741E084
:105D50008D81811101C040E06C818B810E94B90F5F
:105D600086CD809152039091530320E03CE7892B2C
:105D700071F720E030E0EBCF4AE150E06FEF70E0E8
:105D8000CE0107965ED5809152038983EA821B82F9
:105D900082E08C8387E08D8375CD81E090E09093E5
:105DA0009D0380939C0382E390E090933D03809356
:105DB0003C030E94B80C90933B0380933A0357CD69
:105DC000E114F10481F1D0903E03C0904C030091A6
:105DD0003A0310913B030E94B80C801B910B85364F
:105DE000910540F1C7FE26C0D2FE24C00E94B80C27
:105DF00090933B0380933A0380913C0390913D0341
:105E0000019790933D0380933C03892B61F410929A
:105E10009D0310929C0381E090E090935303809344
:105E20005203E12CF12C809152038983EA82809104
:105E30003C030DCD82E390E090933D0380933C03BF
:105E4000F2CF109253031092520311CD40E250E072
:105E50006FEF70E0F6D40BCD2B81273071F0283036
:105E600049F1211104CD2FE1DC011D922A95E9F7BA
:105E700088E08C8383E088A3FACC2C8166E0CE0195
:105E80008196FC01362F11923A95E9F7283080F47B
:105E9000629FB0011124675E7C4F46E050E0D8D489
:105EA00080E0898386E0FE01B196DE011296F3CE92
:105EB0008FEFF7CF6C8186E0FE013596DE0191967B
:105EC00001900D928A95E1F789A19AA181154CE77D
:105ED000940741F42091520330915303232B11F482
:105EE00080E090E09AA389A38BA19CA181155CE737
:105EF000950741F42091520330915303232B11F461
:105F000080E090E09CA38BA38FEF683060F486E084
:105F1000689FB0011124675E7C4F46E050E0CE01DF
:105F20008196E5D480E089830E94B217A0CC80914D
:105F30000C03811509F4C2CA90E199BD09BD09B4E9
:105F400000FEFDCF8091D8008F7D8093D800809196
:105F5000E00082608093E0008091E00081FDFCCF52
:105F60000E943A10ABCA1F921FB61F9211248F9342
:105F70009F93AF93BF9380910B03811113C08091C6
:105F80006A0290916B02A0916C02B0916D024196F1
:105F9000A11DB11D80936A0290936B02A0936C02C5
:105FA000B0936D02BF91AF919F918F911F901FBED3
:105FB0001F90189578941F921FB61F9211248F93EB
:105FC0009F93AF93BF9380916A0290916B02A091CF
:105FD0006C02B0916D020196A11DB11D80936A0201
:105FE00090936B02A0936C02B0936D02BF91AF913E
:105FF0009F918F911F901FBE1F9018951F920F9217
:106000000FB60F9211242F933F934F935F936F938B
:106010007F938F939F93AF93BF93EF93FF93809161
:10602000E10082FF09C08091E20082FF05C08091FB
:10603000E1008B7F8093E1008091DA0080FF24C033
:106040008091D80080FF20C08091DA008E7F8093FD
:10605000DA008091D90080FFA9C080E189BD82E18A
:1060600089BD09B400FEFDCF81E080935403809187
:106070005902811109C00E94C40D0E94210E809115
:10608000E20084608093E2008091E10080FF1AC00A
:106090008091E20080FF16C08091E2008E7F8093A5
:1060A000E2008091E20080618093E2008091D8005C
:1060B00080628093D80019BC85E08093540383E00C
:1060C000809315018091E10084FF2FC08091E20050
:1060D00084FF2BC080E189BD82E189BD09B400FE47
:1060E000FDCF8091D8008F7D8093D8008091E10012
:1060F0008F7E8093E1008091E2008F7E8093E200AA
:106100008091E20081608093E200809158028115C5
:1061100009F452C084E08093540380915403843086
:1061200009F052C082E0809315018091E10083FF65
:106130002CC08091E20083FF28C08091E100877F1E
:106140008093E10082E08093540310925802809182
:10615000E1008E7F8093E1008091E2008E7F80934A
:10616000E2008091E20080618093E20042E060E022
:1061700080E00E94F10D8091F00088608093F00033
:1061800081E08093150180931401FF91EF91BF91FD
:10619000AF919F918F917F916F915F914F913F91BF
:1061A0002F910F900FBE0F901F90189519BC109251
:1061B00054031092590268CF8091E30087FF02C018
:1061C00083E0A9CF81E0A7CF81E0ADCF1F920F92EE
:1061D0000FB60F921124EF92FF920F931F932F93FC
:1061E0003F934F935F936F937F938F939F93AF935F
:1061F000BF93CF93EF93FF9309EE10E0F8018081F6
:10620000C091EC008F70C795CC27C795C82B108222
:1062100080EFE82EF12CF7018081877F80837894CE
:106220000E946110F8011082F701808188608083EC
:10623000CF70F801C083FF91EF91CF91BF91AF91E3
:106240009F918F917F916F915F914F913F912F918E
:106250001F910F91FF90EF900F900FBE0F901F9026
:1062600018958EE1489B02C08A95E1F7489BFECFC6
:106270000895589880E28A95F1F7589A0895FC019C
:106280002BE02A95F1F728E090E080E031E040E152
:106290004A95F1F7880F489B02C08160932742E03E
:1062A0004A95F1F7000040E14A95F1F72A9579F710
:1062B00020E12A95F1F729B132E03A95F1F7000093
:1062C00040E14A95F1F7217092272081920F908347
:1062D0000895A1E0B0E0EEE6F1E375C119828C010A
:1062E0007C01E60EF11CBDDFCE010196C8DFF8018E
:1062F00081938F01EE15FF05B1F781E0998191112E
:1063000080E02196E6E07BC1509A589A0895509813
:10631000589AE89AE9E6F0E080818C7F80830895BE
:106320006150770B91E001C0990F6A95EAF7692FE8
:1063300090E021E0611108C0911599F0589A80E22F
:106340008A95F1F758980895362F3823311539F08A
:10635000589A922730E23A95F1F76695EBCF589824
:10636000F9CF5898ECCFFF920F931F93CF93DF9301
:10637000EC018C01060F111DF9907BDF68E08F2D79
:10638000CFDFC017D107C1F7CDB7DEB7E5E038C121
:106390001F920F920FB60F9211240F931F932F93FA
:1063A0003F934F935F936F937F938F939F93AF939D
:1063B000BF93EF93FF93CF93DF930F92CDB7DEB7E9
:1063C00019824FDFCE0101965ADF082F06950695F8
:1063D0000695982F92959570202F2570920F292F52
:1063E000237096959695920F982797708981892B9F
:1063F000811509F058C0083008F055C080E18A9531
:10640000F1F7589A509A82E08A95F1F700C05898AF
:1064100088E0089F80011124D801A85CBE4F169621
:10642000ED91FC9117973097A9F06091D30170918D
:10643000D40114962D913C911597260F371F119674
:106440008D919C911297680F791F13964C91139719
:106450008C910995F801E85CFE4F6381611549F064
:106460002091D3013091D40184819581820F931FB3
:106470007ADFFFDE80E18A95F1F758985098589AB4
:1064800080E18A95F1F7F801E85CFE4F60816115C3
:1064900049F02091D3013091D40181819281820F02
:1064A000931F17DFDEDE0F90DF91CF91FF91EF9109
:1064B000BF91AF919F918F917F916F915F914F911C
:1064C0003F912F911F910F910F900FBE0F901F9032
:1064D00018950F931F93CF93DF938C0108970CF0BF
:1064E0005EC0F894509A589885E08A95F1F70000BC
:1064F000C02FC695C570802F8570C80F8C2F8370F4
:10650000C695C69593E0000F111F9A95E1F7C80F45
:10651000C8018C2BEC01ADDE00C068E08C2F00DFE1
:1065200090E19A95F1F75098589A489B31C087E0CE
:1065300090E048992FC0F801E85CFE4F6381611537
:1065400059F02091D3013091D40184819581820F3B
:10655000931FBFDE811501F184DE80E28A95F1F799
:106560005898509A90E19A95F1F7F801E85CFE4F3F
:106570006081611549F02091D3013091D40181816E
:106580009281820F931FEFDE74DE789481E008C061
:1065900000C0CBCF019749F4509A589A789480E084
:1065A000DF91CF911F910F91089500C0C2CF2F921C
:1065B0003F924F925F926F927F928F929F92AF9293
:1065C000BF92CF92DF92EF92FF920F931F93CF93E0
:1065D000DF93CDB7DEB7CA1BDB0B0FB6F894DEBF77
:1065E0000FBECDBF09942A88398848885F846E849D
:1065F0007D848C849B84AA84B984C884DF80EE80E7
:10660000FD800C811B81AA81B981CE0FD11D0FB6EF
:10661000F894DEBF0FBECDBFED010895992778E055
:10662000880F991F961708F0961B881F7A95C9F74F
:1066300080950895AA1BBB1B51E107C0AA1FBB1F71
:10664000A617B70710F0A61BB70B881F991F5A95FE
:10665000A9F780959095BC01CD01089597FB072E71
:1066600016F4009406D077FD08D0E4DF07FC05D0CF
:106670003EF4909581959F4F0895709561957F4F59
:106680000895EE0FFF1F0590F491E02D0994082E58
:10669000817006940694811D0694811D0694811DC7
:1066A0000694811D0694811D0694801D0895692716
:1066B0009627692778278727782708957DD1332360
:1066C00012F48A1B9B0B01C077D1B7FF0895821B80
:1066D000930B0895002E083090F0982F872F762F77
:1066E000652F542F432F322F22270850F4CF220F2B
:1066F000331F441F551F661F771F881F991F0A9558
:10670000B2F7002D089597FD1094002E083098F0F0
:106710000850232F342F452F562F672F782F892F7E
:10672000912DF4CF15949795879577956795579503
:106730004795379527950A95AAF71124002D0895B6
:106740008F929F92AF92BF92CF92DF92EF92FF9281
:10675000CF93DF93EC01688179818A819B816115F8
:1067600071058105910521F464E279ED8BE597E0EF
:106770002DE133EF41E050E0D1D049015A019B01B6
:10678000AC01A7EAB1E4E6D06B017C01ACEEB4EF5A
:10679000A5019401EBD0DC01CB018C0D9D1DAE1D3C
:1067A000BF1DB7FF03C00197A109B0488883998333
:1067B000AA83BB839F77DF91CF91FF90EF90DF900B
:1067C000CF90BF90AF909F908F900895B9CF80E009
:1067D00091E0B6CFA0E0B0E080930001909301017A
:1067E000A0930201B09303010895FB01DC0102C0F4
:1067F00005900D9241505040D8F70895FC0141504A
:10680000504030F001900616D1F73197CF0108952E
:10681000882799270895FB01DC0104C08D91019020
:10682000801921F441505040C8F7881B990B0895F6
:10683000FB01DC0102C001900D9241505040D8F79D
:106840000895DC0101C06D9341505040E0F7089578
:10685000DC01CB01FC01F999FECF06C0F2BDE1BD20
:10686000F89A319600B40D9241505040B8F708950F
:10687000F999FECF92BD81BDF89A992780B5089508
:10688000A6E1B0E044E050E0E5CFA8E1B0E042E0AE
:1068900050E0E0CFDC01A40FB51F4150504040F064
:1068A000CB01840F951F2E9105D041505040D8F751
:1068B0000895262FF999FECF92BD81BDF89A0197D0
:1068C00000B4021639F01FBA20BD0FB6F894FA9A38
:1068D000F99A0FBE08950396272FECDFEADF252FE4
:1068E000E9DF242FE7CF0196272FE4DFE2CFDC0199
:1068F000CB0102C02D9105D041505040D8F70895EA
:10690000262FF999FECF1FBA92BD81BD20BD0FB6CB
:10691000F894FA9AF99A0FBE01960895052E97FBFE
:1069200016F400940FD057FD05D024D007FC02D0F8
:1069300046F408C050954095309521953F4F4F4FF4
:106940005F4F089590958095709561957F4F8F4F1B
:106950009F4F089531D0A59F900DB49F900DA49F97
:10696000800D911D11240895B7FFF4CFF3DF821B32
:10697000930B0895A1E21A2EAA1BBB1BFD010DC0AB
:10698000AA1FBB1FEE1FFF1FA217B307E407F507DF
:1069900020F0A21BB30BE40BF50B661F771F881FBB
:1069A000991F1A9469F760957095809590959B0151
:1069B000AC01BD01CF010895A29FB001B39FC001FA
:1069C000A39F700D811D1124911DB29F700D811D1B
:1069D0001124911D0895F894FFCF3E1164116A119E
:1069E00064116A11BC11DD116A11E312F0127F1EED
:1069F0009B1E9F1EA31EA71EAB1EAF1EB31EB71E5F
:106A0000BB1EBF1E352E502E572E882E9F2EBC2EFD
:106A1000CD2EE02E212F262F372C372C372C2C2F44
:106A2000252C292C5C2C682C732C7E2C812CB52CCD
:106A3000D72C222C202EDE2CE12CE42C102D4C2DDA
:066A40004E2D502D842DA7
:106A46000100000001010201191A1B1C1D1E1F2056
:106A56002122000001000010001010F6F5F4F1F0FC
:106A6600373392939594313267349701B50C260FDC
:106A7600190D1A0D3C0F1D0F00000001000000004B
:106A86000000000A01000000000000010B000000E9
:106A9600000000080C0000000000000000000908CB
:106AA60004140000000000000B18000000000000A5
:106AB600333236349700F1F0F4F5F69567933700E4
:106AC60071E434629C8E3168004422320001DE009B
:106AD600AC0006021F023F02000102020202060685
:106AE600060909090909090F0F0F0F0F0F151515CB
:106AF60018191919191919191919192324252525C8
:106B060025252500FF0100010000FFFF0000010010
:106B160001FF007103E200E900EA00B500B600B724
:106B260000CD008301CC008A019201940121022349
:106B36000224022502260227022A02B300B4006FAD
:106B46000070009F01CB019F02A002E200E900EA6B
:106B560000B500B600B700CD008301CC008A0192D3
:106B66000194012102230224022502260227022A79
:106B760002B300B4006F0070009F01CB019F02A01A
:026B860002000B
:00000001FF
